:020000040800F2
:10000000200C00208D0100083147000891470008AE
:10001000090100080B0100080000000000000000BA
:100020000000000000000000000000000F010008B8
:10003000110100080000000013010008B953000876
:1000400000000000000000000000000000000000B0
:1000500000000000000000000000000000000000A0
:100060000000000000000000000000000000000090
:100070000000000000000000000000000000000080
:100080000000000000000000000000000000000070
:100090000000000000000000000000000000000060
:1000A0000000000000000000000000000000000050
:1000B0000000000000000000000000000000000040
:1000C0000000000000000000000000000000000030
:1000D0000000000000000000000000000000000020
:1000E0000000000000000000000000000000000010
:1000F0000000000000000000000000000000000000
:10010000883B0008FEE7FEE7FEE7FEE7FEE7FEE7C6
:10011000FEE7FEE7FEE72020174D01202968014396
:100120002960361F37602F4600B500BF3D680220AA
:100130000540FBD01120114908601148786000206B
:10014000F862104839680143396000BF3D680E48C5
:100150000540FBD03D1D0C3E032131600221716042
:10016000B7602F4601F000FC7D680C200540082D8B
:10017000FAD180CE00BD01BC001002400020024038
:1001800000801004000000010000000200B500BF64
:10019000104D85F30888104D85F30988022585F3F5
:1001A0001488BFF36F8F0D4E0D4DAB460D490E48B1
:1001B0000D6805430D600D490D480D6885430D60C0
:1001C000FFF7AAFF0B48056801200543A847DFE7B2
:1001D00000BD0000200C0020200E0020040F002095
:1001E000100F00201410024014007E00281002405E
:1001F00000007E0000010008040F0020200E0020F7
:1002000000000000000000000000000000000000EE
:100210000A0000000000000000C0000800C0000844
:10022000B8100020481000209715A06D00000000B5
:10023000C3414E4431680F40361D70470000000036
:10024000C24F522031680F43361D70470000000036
:10025000C3584F5231684F40361D704700000000B0
:10026000C6494E5645525420FF43704700000000D7
:10027000C2303D20002F01D0002701E001277F423E
:100280007047000000000000C3303C3E002F01D149
:10029000002701E001277F4270470000700200083C
:1002A000C2303E20002F01DC002701E001277F4201
:1002B00070470000A0020008C2303C20002F01D48B
:1002C000002701E001277F42704700000000000086
:1002D000C13D20203068874201D0002701E001277E
:1002E0007F42361D70470000D0020008C23C3E200D
:1002F0003068874201D1002701E001277F42361D87
:100300007047000000000000C13C20203068874298
:1003100001DC002701E001277F42361D7047000005
:1003200060020008C13E20203068874201DB0027C0
:1003300001E001277F42361D70470000EC020008F3
:10034000C23C3D203068874201DA002701E00127E6
:100350007F42361D7047000000000000C23E3D2075
:100360003068874201DD002701E001277F42361D0A
:100370007047000000000000C2553E2030688742F0
:1003800001D3002701E001277F42361D704700009E
:1003900078030008C2553C203068874201D8002706
:1003A00001E001277F42361D7047000094030008DA
:1003B000C344303C002F01D4002701E001277F42D5
:1003C000361D7047B0030008C344303D31680F4309
:1003D000002F01D0002701E001277F42361D704722
:1003E00000000000C2443D2007CE3B1C0027801ABD
:1003F0008B41384300D1FF43704700005C03000885
:10040000C34D494E01CE874200DD074670470000CC
:1004100000040008C34D415801CE874200DA074668
:100420007047000008030008C657495448494E2049
:1004300030683F1A716830680D1AAF4201D8002742
:1004400001E001277F42083670470000B80200082B
:10045000C64C534849465420384680CE87407047A2
:1004600000000000C652534849465420384680CE0A
:10047000C740704764040008C74152534849465476
:10048000384680CE0741704700000000C7455845F8
:10049000435554450120384380CE00470121704622
:1004A0008843026810470000391C80CEF6D07046A1
:1004B000001D004701CEB84201D180CEF7E70746C4
:1004C000ECE700000099491C0091E7D703B0EEE784
:1004D0000099C919009180CEE0D703B0E7E700008A
:1004E00002CE0124E40773465B1E1A680919781AC4
:1004F00007B480CEDBE7000002CEB942F1D180CE56
:10050000CCE7000040020008C54C4541564520207C
:1005100002B000BD00000000C63F4C4541564520DA
:100520003F1C80CE00D1704702B000BD000000002B
:10053000C1492020361F3760009F01983F1870473F
:1005400050020008C14A2020361F3760039F0498DC
:100550003F18704744050008C6554E4C4F4F502079
:1005600003B07047E4030008C3533E44FD17361F31
:1005700037602F467047000024030008C24D2B202F
:1005800003CEFA17C91950410746361F316070472C
:1005900088020008C2312B207F1C70479405000898
:1005A000C2312D207F1E70478C040008C12B2020F3
:1005B0003068361D3F18704740030008C12D2020C9
:1005C0003068361DC71B704730020008C64E4547CD
:1005D000415445207F42704768050008C2442B20E3
:1005E00007CE80184F41361F30607047DC05000889
:1005F000C2442D2007CE101AB9410F46361F306075
:100600007047000058050008C7444E45474154450F
:10061000306800214042B9410F4630607047000009
:10062000F0050008C73F4E45474154453F1C80CE6A
:1006300000D57F4270470000CC050008C3414253FB
:10064000002F00D57F42704778040008C44441421F
:10065000532020203F1CDBD470470000C803000853
:10066000C344322A306800187F4130607047000070
:1006700060060008C344322F306840107F10894163
:10068000C90708433060704708060008C12A2020C7
:1006900031684F43361D70474C060008C3554D2A3C
:1006A0003846316840B40A04120C0B0C0404240CC4
:1006B000050C164666431F466F4318466043010CFF
:1006C000000436184F4128465043010C00043618E8
:1006D0004F41354640BC3560704700007C0500083E
:1006E000C24D2A2035687D4000B520B4002F00D5CA
:1006F0007F423568002D00D56D423560FFF7D0FF91
:1007000020BC002D01D5FFF783FF00BD8C0600083B
:10071000C6554D2F4D4F442001CE31682024002274
:100720004918404113465341C01B5B4101D0491C4D
:1007300000E0C019641EF3D10F463060704700001E
:1007400000000000C6534D2F52454D2000B53068C3
:1007500001B480B480CEFFF77DFF009D002D00D551
:100760006D42361F37602F46FFF7D6FF20BC009C36
:100770006C40002C00D57F4220BC002DEFF30080A0
:1007800001B430683760074601BC80F3008800D5AB
:100790007F4230683760074600BD0000A0050008B2
:1007A000C42F4D4F4420202000B580B43168CF17AE
:1007B00020BC361F37602F46FFF7C8FF00BD000082
:1007C00014040008C12F202000B580B43168CF1771
:1007D00020BC361F37602F46FFF7B8FF361D00BD1F
:1007E000C4070008C34D4F4400B5FFF7DDFF80CEBE
:1007F00000BD0000A0070008C64D552F4D4F4420F6
:1008000000B580B4009F361F00213160FFF784FFE0
:1008100020BC80B42F46FFF77FFF20BC361F376017
:100820002F4600BDAC050008C6464D2F4D4F442055
:1008300000B580B435687D40002D01D4002501E06D
:1008400001256D4220B4FFF781FF20BC31680D40C7
:1008500005D07F1E20BC30682D18356000E001B047
:1008600000BD000074060008C2552F20361F00216D
:10087000316000B5FFF750FF361D00BDE0060008EF
:10088000C24D2F2000B5FFF761FF361D00BD0000EF
:1008900080080008C52A2F4D4F44202000B580B4A1
:1008A00080CEFFF71FFF20BC361F37602F46FFF7B3
:1008B0004DFF00BD28080008C22A2F2000B5FFF711
:1008C000EDFF361D00BD000008050008C34E49506D
:1008D000361D70479C060008C45455434B20202009
:1008E000361F716831607760704700003C06000871
:1008F000C45049434B202020BF00F75970470000E7
:1009000024060008C4524F4C4C202020B800002878
:1009100001DC80CE70473758011F72583250081CD6
:10092000FAD1361D7047000018050008C3524F5415
:100930003D4677683168716035607047CC080008C3
:10094000C42D524F542020203D46376871683160D5
:1009500075607047E4070008C23E522080B480CE24
:1009600070470000F0080008C2523E20361F376072
:1009700080BC704768090008C2524020361F3760AB
:10098000009F70472C090008C3323E5203CE01B4C9
:1009900080B40F1C7047000088090008C332523E23
:1009A00003BC083E31607760074670479C09000829
:1009B000C332524000980199083E31607760074683
:1009C0007047000068080008C45357415020202099
:1009D0003068376007467047C8090008C34455505F
:1009E000361F376070470000F8070008C44F5645AF
:1009F00052202020361F376077687047D8080008DB
:100A0000C444524F5020202080CE70470409000873
:100A1000C432445550202020083EB16831607760D0
:100A200070470000DC090008C5324F5645522020AF
:100A3000083E316931607760F7687047280A00081E
:100A4000C53244524F502020776808367047000066
:100A5000400A0008C5325357415020207068776023
:100A60000746B0683168B16030607047EC09000833
:100A7000C43F445550202020002F01D0361F37603E
:100A800070470000100A0008C3535040361F3760FB
:100A900037467047880A0008C35350213E4680CE2F
:100AA00070470000B0090008C3525040361F37603D
:100AB0006F467047A80A0008C3525021BD4680CE39
:100AC0007047000044070008C544455054482020A2
:100AD00000B501F0ADFA3F68361F37603746316820
:100AE000CF1B3F1FBF10361D00BD0000000A0008CD
:100AF000C5434F554E5420207D1C3F78361F35602E
:100B000070470000980A0008C72F535452494E47B7
:100B10003168CD1B70683F1877602F46361D7047CF
:100B2000540A0008C4534B495020202003CE401CD7
:100B3000401E04D00A78BA4201D1491CF8E7361F9A
:100B40003160074670470000240B0008C45343413E
:100B50004E20202003CE401C401E04D00A78BA420A
:100B600001D0491CF8E7361F316007467047000086
:100B7000B80A0008C2533D2003CE3F1C07D00278BC
:100B80000B78401C491C9A4201D17F1EF7D102D13B
:100B900001277F4200E00027704700003005000871
:100BA000C7434F4D504152457168CD1B00B520B42D
:100BB00071688F4200DB0F1C31687160361D00BF09
:100BC000002F23D075682D78346824782C1B002CD6
:100BD000EFF3008001B4361F71683160B168716055
:100BE000B760274601BC80F3008804D001B080B410
:100BF0000027361D09E037687F1C75686D1CB068DA
:100C0000441E7760B5602746361DD9E780BC002FAB
:100C1000EFF3008001B4083601BC80F3008807D0F0
:100C2000002F01D4002701E001277F420120074364
:100C300000BD202000B5B16802B4716802B431680B
:100C400002B480B480B0484601B4E946F768103673
:100C50004D462D694C46E4684B465B68E31A5B1CC5
:100C60005B19083E336077602F4600BFFFF744FCF6
:100C7000DF0C0008009D019805442D784C46A468BF
:100C80002478AC4226D1009D019805444C46A468C6
:100C90004B465B680C3E34607560B7601F46FFF7DB
:100CA0006BFF002F80CE15D0009D019805444C4667
:100CB000E468009B019803444A4612699A1AA21AF2
:100CC00003B00C3E32607560B7600B4F01BC8146CB
:100CD00004B000BD0098401C0090CBD703B04D4637
:100CE0002D694C46E4680C3E34607560B76000279F
:100CF00001BC814604B000BDFFFFFFFFC80A000829
:100D0000C6534541524348207068874200B502DD12
:100D10000027361D00BD002F02DC064F361D00BD2A
:100D20007068002802DC0027361D00BDFFF782FF37
:100D300000BD0000FFFFFFFFF00A0008C5434D4F54
:100D4000564520203B1C83CE00D17047021C0A432D
:100D50001A430324144006D10A680260091D001DCD
:100D60001B1FF9D170470A780270491C401C5B1E9A
:100D7000F9D17047000D0008C6434D4F56453E203F
:100D80003B1C83CE00D17047C018C918021C0A430F
:100D90001A430324144006D1091F001F0A68026089
:100DA0001B1FF9D17047491E401E0A7802705B1E56
:100DB000F9D1704740090008C44D4F564520202006
:100DC00000B580B4316870680F1A009DBD4280CEB6
:100DD00006D920BC361F37602F46FFF7D1FF05E04C
:100DE00020BC361F37602F46FFF7ACFF00BD000068
:100DF0003C0D0008C3555043612F00B503DB7A2F2B
:100E000001DCDF20074000BDA00B0008C555505095
:100E10004552202030683F1830683760074600B5DB
:100E2000FFF76AFB4F0E0008009D019805442D78DE
:100E3000361F37602F46FFF7DFFF009D01980544FE
:100E40002F7080CE0098401C0090EDD703B000BDFD
:100E5000740B0008C5504C414345202000B5306854
:100E600001B480B47F1C306837600746FFF7A8FFE5
:100E700020BC10BC2C7000BD0C0E0008C446494CB0
:100E80004C2020203A1C83CE002803D00A70491C35
:100E9000401EFBD1704700007C0E0008C545524142
:100EA00053452020361F3760002700B5FFF7EAFFC3
:100EB00000BD0000B80D0008C14020203F68704709
:100EC000780D0008C25740203F887047540E000834
:100ED000C24340203F78704750040008C1212020C1
:100EE000306838607768083670470000C40E000824
:100EF000C257212030683880776808367047000074
:100F0000D00E0008C2432120306838707768083658
:100F100070470000B80E0008C24F4E20012040422A
:100F2000386080CE70470000DC0E0008C34F464694
:100F30000020386080CE704728040008C4494E4322
:100F4000522020203868401C386080CE7047000056
:100F5000F40D0008C4444543522020203868401E48
:100F6000386080CE704700003C0F0008C22B212063
:100F700030683968091839607768083670470000AA
:100F800078090008C232402003CF361F074631607F
:100F900070470000840F0008C23221203A1C83CE23
:100FA00003C270472C0F0008C44E4F4F5020202022
:100FB00070470000700A0008C54E414D453E202094
:100FC000361F376000B500F0E5FF1F20074030688E
:100FD0003F183F1D03218F43361D00BDB80F000889
:100FE000C53E4E414D45202001218F4300B500BF35
:100FF0003F1F361F376000F0E1FF8020074080CEA2
:10100000F6D000BD00B500BF00F0D8FF002F2BD0F8
:101010003D781F2005403068854223D17D1C0C3E61
:10102000316931607560B760F768FFF7A5FD002F83
:1010300080CE17D07760361DFFF7C2FF35682D7858
:1010400040200540EFF3008001B4361D01BC80F361
:10105000008803D0361F3760054F02E0361F376027
:10106000012700BD3F1FCFE70027083600BD000065
:10107000FFFFFFFFA80F0008CF5345415243482D03
:10108000574F52444C495354002F00B501D10836F4
:101090000CE075682D7830682D183C68641E2C4073
:1010A000641CA400E4192746FFF7ACFF00BD000054
:1010B000F00E0008C54449474954202001CE30387D
:1010C0000BD40A2802DBC01F0A2806DBB84204DA68
:1010D00001277F42361F30607047002770470000AD
:1010E000540F0008C543454C4C2B20203F1D704732
:1010F000E4100008C543454C4C532020BF00704706
:10110000F4100008C543454C4C2D20203F1F70476C
:101110004C0B0008C443454C4C202020361F376040
:10112000042770473D0C361F37602F4600B501F08D
:10113000A7F901F0A5F900BD31680D0C083E356036
:10114000776000B500F04EFFBF1C00F04BFF00BD04
:101150003D882D04BF1C361F356000B500F024FF0C
:1011600031680F43361D00BD30680740002F01D0A5
:10117000002701E001277F423068002801D40025C4
:1011800001E001256D427D402F46361D704720202D
:101190003F1D3168CF1B7F10154D3D40FC0A15489F
:1011A000044024042C43083E37607460B760124F3B
:1011B00000B5FFF7D9FF1148074031680F43361FCC
:1011C000B168316077600E4FFFF7CEFF0D480740E2
:1011D00031680F437068002801D4002501E0012523
:1011E0006D42094805403D432F46083600BD0000CA
:1011F000FF070000FF0300000000200000200000A7
:1012000000004000000800000000000400B5FFF7E7
:10121000BFFF0148074300BD00D000F0361F376014
:10122000024F00B501F02CF900BD000000B5000030
:10123000361F3760024F00B501F022F900BD0000F3
:1012400000BF0000361F71683160776000B5FFF79E
:10125000DDFF306837600746FFF76EFF00BD2020D6
:10126000361F3760044F00B501F00AF9361F3760AA
:10127000024F01F005F900BD361F00003760000085
:10128000361F3760074F00B501F0FAF8361F376098
:10129000054F01F0F5F8361F3760044F01F0F0F804
:1012A00000BD000070460000401E000007680000FE
:1012B00000B501F033F8FFF7A9FFFFF733FF00BDDA
:1012C00000B501F02BF80220074080CE01D0FFF7D7
:1012D000AFFFFFF7EDFF00BD00B5FFF79FFF00BDBB
:1012E000361F37607046401E0768401D00470000EB
:1012F000361F3760009F7F1E3978C919091D0322E8
:101300009143491C0091704704110008C7414C49A2
:10131000474E4544FF1C03218F437047361F3760FB
:101320007046401E076800BD10070008C8434F4DB7
:1013300050494C452C20202000B5FFF7B9FF00BDD7
:10134000E00F0008C53E424F4459202001218F4341
:10135000BF68704700B5FFF76BFFFFF75FFF361FF1
:101360003760024FFFF7A4FF00BD00001C13000808
:1013700000B501F03DF801F02DF9FFF7EBFF306803
:101380003760074601F06CF801F03EF800BD202000
:1013900000B520BC01218D43361F37602F4601F078
:1013A0008BF8FFF70DFE3F1DFFF74CFF00F0BAFD75
:1013B00000BD000000B500BF00F0BEF80010002026
:1013C000B8080008C3494D4D024901204042086059
:1013D00070470000001000202C130008813A2020E4
:1013E00000B501F0A1FE01F06BFE01F0F3F801F091
:1013F0006BF802F08FF8FFF76FFF00BD180F0008C1
:10140000C73A4E4F4E414D4500B501F059FE00F030
:1014100061FD01F017F800F081FF00F0E9FE30688F
:1014200038600027361D01F01BF800F077FF02F04E
:1014300071F8FFF751FF00BDB410000885444F4517
:10144000533E2020361F3760044F00B5FFF774FF6E
:10145000FFF706FFFFF714FF00BD00009013000820
:101460003C140008C64352454154452000B500F0E5
:10147000D1FF00F0BDFF30683760074601F0AAF8E1
:10148000FFF768FF01F008F900F0BEFF00BD0000A3
:1014900044130008C73C4255494C445300B5FFF77C
:1014A000E5FF00BDDC130008C8434F4E5354414EC6
:1014B0005420202000B5FFF75BFFFFF769FF361FC0
:1014C00037607046401E076800BD00000C1300081E
:1014D000C345515500B5FFF7EDFF00BDA814000846
:1014E000C932434F4E5354414E54202000B5FFF7AC
:1014F0003FFF00F0B5FFFFF74BFF083E77607046F7
:10150000401E07684168316000BD0000BC0500084E
:10151000C85641524941424C4520202000B500F0B8
:1015200045FF00F027FFFFF723FF361F3760042732
:1015300000F02EFFFFF72CFF361F37607046401E6D
:10154000076800BD64140008C74255464645523A34
:1015500000B500F02BFF00F00DFFFFF7ABFF00F030
:1015600017FF00BD48150008C455534552202020E0
:1015700000B5FFF7FDFEFFF70BFF361F3760704623
:10158000401E07685F4400BD7047000068150008F2
:10159000C54445464552202000B500F007FF00F045
:1015A000E9FEFFF7E5FE361F3760042700F0F0FE86
:1015B000FFF7EEFE7046401E0068016801221143ED
:1015C00008BC9E460847000000B500BFFFF7B4FF07
:1015D0000410002000B500F0F9FD3F68002F80CE18
:1015E00005D080CEFFF76CFE00F03AFF05E03D46E7
:1015F0007768083601200543A84700BD00B500F014
:1016000053FE01F085F81E496E76616C6964206FA7
:1016100070657261746F7220666F7220746869738E
:101620002074797065000000361F3760014F01F0AB
:101630009DF800BDF3FFFFFF7146491E0868491D74
:101640008E46076080CE7047361F37607146491E50
:101650000868491D8E46076870470000E0140008BE
:10166000C556414C5545202000B5FFF7ADFE80B46E
:1016700080CE00F09BFE00F07DFEFFF779FE20BCDF
:10168000361F37602F4600F075FE3068386004273B
:10169000361D00F07DFEFFF77BFE361F376070467B
:1016A000401E076811480568104900200860002D99
:1016B000EFF3008001B4361F37602F4601BC80F382
:1016C000008806D1361F0A4F0A493160FFF782FFB2
:1016D0000BE0012F06D1361F074F08493160FFF795
:1016E00079FF02E0FFF78AFF80CE00BD04100020E2
:1016F000BC0E000848160008E00E00083816000866
:10170000080B000882544F200120014908607047EF
:101710000410002000B500F001FE361F37600427DA
:1017200000F018FE00BD202000B500F0F7FD0120FC
:10173000074330683760074600F05EFC00BD20209C
:1017400000B500F0EBFD00BD0120074300B500F03F
:1017500087FE00BD361F3760034F00B5FFF7B0FDB1
:10176000FFF7F2FF00BD00009C040008361F376041
:10177000034F00B5FFF7A4FDFFF7E6FF00BD000033
:10178000A8040008361F3760034F00B5FFF798FD27
:10179000FFF7C0FF00BD00009C040008361F376043
:1017A000034F00B5FFF78CFDFFF7B4FF00BD00004D
:1017B000A8040008361F3760034F00B5FFF780FD0F
:1017C00000F04EFE00BD0000E0120008361F37603A
:1017D000024F00B5FFF7B0FD00BD0000080A000889
:1017E000361F3760024F00B500F04AFE00BD000012
:1017F00000BD0000361F3760044F00B5FFF760FDE5
:10180000FFF788FFFFF79CFF00BD0000E004000821
:10181000361F3760044F00B5FFF752FDFFF77AFF20
:10182000FFF78EFF00BD0000F8040008361F376088
:10183000044F00B5FFF744FDFFF786FFFFF774FF85
:1018400000BD0000C4040008361F3760044F00B517
:10185000FFF736FDFFF778FFFFF766FF00BD0000DA
:10186000D004000800B500BFFFF766FE0810002096
:1018700005480568361F37602F4600B5FFF760FF43
:1018800001490F6080CE00BD08100020361F376070
:10189000034F00B5FFF714FDFFF73CFF00BD00004C
:1018A000B404000800B5FFF76DFF306837600746E5
:1018B000FFF73AFF00BD202000B500BF361F37609C
:1018C000374600F073FC3F6830688742EFF30080D2
:1018D00001B47768083601BC80F3008802D0FFF7B6
:1018E00023FFEBE700BD202000B5FFF76FFFFFF7F8
:1018F000E3FF02490F6080CE00BD00000810002009
:1019000000B5FFF74BFF00BD040F0008C55041555F
:101910005345202000B500BFFFF74CFE0C100020FF
:1019200004170008C244492072B670471411000819
:10193000C245492062B670476C0F0008C25B49205F
:10194000EFF3108072B601B4704700006016000813
:10195000C2495D2001BC80F3108870479C0E0008CE
:10196000C75345544D41534B3D683068C4432C40E8
:10197000706804433C60B7680C367047580900082B
:10198000C7494E49542D494F00B500BF3D68002D51
:1019900004D03D687C682C600837F7E780CE00BD36
:1019A00090150008CA4F4646543252454C323520F5
:1019B000BD0E0120054000B520B40F4D3D406D0027
:1019C0003C0C0E48044024032C43FD0A0120054032
:1019D000009B6B40012043409B0523437F0B01206C
:1019E0000740009D7D4001204540ED051D4380BC22
:1019F0003F067F422F4300BDFF070000FF030000AA
:101A0000980F0008C63E424445535420361F3760A5
:101A100000B5FFF79DFBFFF7CBFF30683F183F1D78
:101A2000361D00BD24190008C4424F522120202039
:101A3000306839780143397077680836704700009C
:101A400030190008C54242494321202030683978C6
:101A500081433970776808367047000060190008C4
:101A6000C842544F47474C452120202030683978E0
:101A7000414039707768083670470000281A00081E
:101A8000C4425453542020203F7831680F40361D03
:101A90007047000078100008C34F52213068396841
:101AA000014339607768083670470000801A0008E3
:101AB000C44249432120202030683968814339607D
:101AC000776808367047000050190008C7544F4720
:101AD000474C45213068396841403960776808369D
:101AE00070470000441A0008C35453543F683168DB
:101AF0000F40361D70470000E81A0008C4435345E4
:101B000054202020306839780143397077680836CE
:101B100070470000FC1A0008C443434C52202020A8
:101B2000306839788143397077680836704700002B
:101B3000601A0008C743544F47474C45306839780E
:101B4000414039707768083670470000181B00085C
:101B5000C4434745542020203F7831680F40002F70
:101B600001D1002701E001277F42361D7047202068
:101B7000074805688020054000B508D0054D064897
:101B8000686006486860802029698143296100BD3A
:101B9000102002400020024023016745AB89EFCDB1
:101BA000083E134931607760124F00B53068451E1A
:101BB000002DEFF3008001B4356001BC80F3008894
:101BC00004D0FD6801200540002DEFD1FD683424CC
:101BD0002C40FC6030680028EFF3008001B42F46F1
:101BE000361D01BC80F3008801D10348074300BDC6
:101BF00000001000002002400000008000B5FFF748
:101C0000B7FF084901200D6805430D603068388032
:101C100077680836FFF7C4FF024901200D68854345
:101C20000D6000BD102002400B483F1A00B5FFF7C1
:101C30009FFF0A4D02202969014329616F614020FD
:101C400029690143296180CEFFF7AAFF04490220D8
:101C50000D6885430D6000BD0000000800200240B3
:101C60001020024000B5FFF7C9FF80CE00BD202044
:101C70003D783068854200B502D17768083600BDEE
:101C80003D4601218D4301200740EFF3008001B460
:101C90002F4601BC80F3008806D031680D023C78E5
:101CA0002C433760274605E07D782D0231680D43CF
:101CB00037602F46306837600746FFF7D3FF00BD17
:101CC000074D31680D40083E3560776000B5FFF77D
:101CD000C9FF31680D0CBF1C3560FFF7C3FF00BDA5
:101CE000FFFF0000083E044931607760034F00B5F4
:101CF000FEF79EFB00BD0000000000080000100879
:101D0000361F376000B5FFF7EDFF002F80CE02D001
:101D1000FFF7AEFF03E0306838707768083600BD23
:101D2000361F376000B5FFF7DDFF002F80CE02D0F1
:101D3000FFF798FF03E0306838807768083600BD09
:101D4000361F376000B5FFF7CDFF002F80CE02D0E1
:101D5000FFF7B6FF03E0306838607768083600BDEB
:101D60003C190008C7464C455241534530683F185E
:101D700030683760074600B5FEF7BEFBC71D000898
:101D8000009D01980544361F37602F46FFF7AAFFD4
:101D9000002F80CE09D0009D01980544361F376082
:101DA0002F46FFF741FF084F07E0009D01980544CB
:101DB00006482860361F376004270098C019009035
:101DC00080CEDDD703B000BD00080000FFFFFFFF9D
:101DD000C4130008C6464C50524F472030683F1885
:101DE00030683760074600B5FEF786FB111E000815
:101DF0003D88009C01980444083E35607760274682
:101E0000FFF730FFBF1C0098801C0090F0D703B094
:101E100080CE00BD083EB1683160776000B5FFF745
:101E2000A5FF31687D1811480468083E346077606A
:101E30002F46FFF785FF30683F1830683760074648
:101E4000FEF75AFB691E00083D68009C0198044497
:101E5000083E356077602746FFF772FF3F1D009808
:101E6000001D0090F0D703B080CE00BD280200080E
:101E700010150008CB434F444552414D425546464C
:101E800000B500BFFFF71BFB0000002000B500BF3E
:101E9000FFF703FC101000200348056803494D1BA1
:101EA000361F37602F4670471010002000000020BA
:101EB00000B500F033FAFFF7EFFF3168CF1B361D96
:101EC00000BD0000041A0008C92B42554646434F86
:101ED0004D5020200C480568002D00B513D10C3E54
:101EE0000A4931600A497160B760FF27FEF7CAFFEF
:101EF000361F3760064F00F011FA3168CF1B0249D8
:101F00000F607768083600BD101000200002000046
:101F100000000020B01A0008C92D42554646434F24
:101F20004D50202009480568002D00B50DD000F067
:101F300089FA361F3760064FFFF7AEFFFFF7B8FF8D
:101F4000FFF74CFF00200149086000BD1010002081
:101F5000000000200B480568002D00B511D0361F89
:101F60003760FFF799FF08497D18361F37602F4605
:101F7000FEF75EFA002F80CE03D002480568ED1907
:101F80002F4600BD1010002000020000181F00089E
:101F9000C343404300B5FFF7DDFF3F7800BD0000BD
:101FA000341B0008C357404300B5FFF7D3FF3F88F9
:101FB00000BD0000981A0008C240432000B5FFF79A
:101FC000C9FF3F6800BD0000901F0008C3432143C4
:101FD00000B5FFF7BFFFFFF793FE00BDA41F000889
:101FE000C357214300B5FFF7B5FFFFF799FE00BDCA
:101FF00094140008C221432000B5FFF7ABFFFFF7A0
:102000009FFE00BD00B500BFFFF796FA1410002038
:10201000501B0008C453454C4620202000B500BF8B
:10202000FFF7ABFA000000000C190008C253302083
:1020300000B500BFFFF7A1FA18000000C81E000895
:10204000C252302000B500BFFFF797FA1C00000015
:1020500014200008C42354494220202000B500BFAA
:10206000FFF78BFA20000000CC1A0008C42754495F
:102070004220202000B500BFFFF77FFA24000000B7
:1020800000140008C33E494E00B500BFFFF775FAC3
:102090002800000080190008C8584F4E2F584F469E
:1020A0004620202000B500BFFFF767FA2C00000093
:1020B000D41D0008C74543484F494E4700B500BFEF
:1020C000FFF75BFA30000000B81F0008C34F5554FB
:1020D00000B500BFFFF751FA34000000CC1F000824
:1020E000C44241534520202000B500BFFFF745FA08
:1020F0003800000000B500BFFFF73FFA3C000000C9
:1021000000B500BFFFF739FA400000005420000876
:10211000C344504C00B500BFFFF72FFA4400000045
:1021200040200008C54F50564543202000B500BF51
:10213000FFF723FA48000000741E0008C5495056F6
:102140004543202000B500BFFFF717FA4C00000000
:1021500000B500BFFFF711FA50000000F41F00089F
:10216000C350414400B500BFFFF707FA98000000D4
:1021700024210008C2424C2000B500BFFFF79FF9A0
:1021800020000000E0200008C244502000B500BF3D
:10219000FFF7D2F91810002074210008C252502015
:1021A00000B500BFFFF7C8F91C10002000B500BF44
:1021B000FFF7C2F9201000206C200008C3584450DB
:1021C00000B500BFFFF7B8F92410002000B500BF2C
:1021D000FFF7B2F92810002000B500BFFFF7ACF9F7
:1021E0002C10002000B500BFFFF7A6F9301000202A
:1021F00000B500BFFFF7A0F93810002000B500BF00
:10220000FFF7D8F93C10002000B500BF00F03FFFF9
:10221000142200084810002000B500BFFFF78CF919
:102220008C1000203C210008C34B45595D46ED6CE5
:102230002D6800B501200543A84700BD940800089B
:10224000C44B45593F2020205D46ED6C6D6800B5BC
:1022500001200543A84700BDA4190008C4454D4905
:10226000542020205D46696B491C69635D46AD6C56
:10227000AD6800B501200543A84700BDD014000893
:10228000C4545950452020205D46696BC9196963C3
:102290005D46AD6CED6800B501200543A84700BD63
:1022A0002C200008C24352205D46002068635D4632
:1022B000AD6C2D6900B501200543A84700BD0000A5
:1022C00080220008C553504143452020361F376007
:1022D000202700B5FFF7C6FF00BD00005C22000804
:1022E000C653504143455320002F00DC0027361FC2
:1022F0003760002700B500BFFEF7FEF80F23000887
:10230000FFF7E4FF0098401C0090F9D703B000BD30
:10231000B4200008C44845524520202003480568E1
:102320002D68361F37602F467047000024100020AC
:10233000CC200008C34F5247024805682F6080CE6A
:10234000704700002410002088210008C5414C4C33
:102350004F542020034805682968C919296080CE98
:10236000704700002410002010210008C552484585
:102370005245202002480568361F37602F467047B7
:102380001C100020C4220008C652414C4C4F54205F
:1023900002490868C019086080CE70471C100020F0
:1023A00088230008C652414C49474E20034805681F
:1023B000ED1C03218D4301490D6070471C10002066
:1023C000A4220008C3524F4D0148024908607047DB
:1023D0001810002024100020C4230008C352414DCF
:1023E00001480249086070471C100020241000209A
:1023F00004480568361F37602F4600B5FFF7E4FF35
:1024000000BD00002410002001490F6080CE7047FD
:1024100024100020064805680648854201D00025A2
:1024200001E001256D42361F37602F4670470000DE
:1024300024100020181000204C230008C5414C49EE
:10244000474E202000B5FFF769FFFF1C03218F4393
:10245000FFF772FF00BD0000641D0008C12C2020A2
:1024600000B5FFF75BFFFFF7C7FD361F3760042796
:10247000FFF770FF00BD0000E0220008C2572C20CB
:1024800000B5FFF74BFFFFF7ADFD361F37600227A2
:10249000FFF760FF00BD0000DC230008C2432C20D2
:1024A00000B5FFF73BFFFFF793FD361F37600127AD
:1024B000FFF750FF00BD202002480568361F376037
:1024C0002F467047381000200448056804490D6005
:1024D0002D1F2D6801490D60704700003810002045
:1024E0008C1000200248056802490D60704700000A
:1024F0008C10002038100020E01F0008C446494E10
:10250000442020207D1C3C78083E356077602746BB
:1025100000B5FEF77FFC3D78002D26D0154D2C46EA
:102520000834083E346077602F4600BFFDF7D8FFBF
:102530006B2500087D1C3C78009B019803441B68B8
:102540000C3E34607560B7601F46FEF79DFD002F9E
:1025500000D180CE04D003B031687160361D00BD5B
:102560000098001D0090E5D703B0361F37600027A4
:1025700000BD00003010002060210008C52E4E4133
:102580004D4520207D1C3F781F200740361F3560B9
:1025900000B5FFF779FEFFF799FE00BD30683F18E0
:1025A00030683760074600B5FDF7A6FFCD25000867
:1025B000009D019805442D78361F37602F46FFF7A0
:1025C0006FFF0098401C0090F2D703B0FFF73AFF6E
:1025D00000BD202000B5FFF77DFC361F37602027A7
:1025E00000F092FC7D1C3F780C3E35607760B56052
:1025F000FEF710FC254805680C3E3760F1687160F5
:10260000B7602F46FEF740FD002F80CE0ED0FEF7BC
:10261000EBFCFFF749FEFFF7B5FF00F079F80D6915
:1026200073207265646566696E656420FFF70AFF52
:1026300035682D78ED191548046823685B1E1D4028
:10264000AD00241D64192568083E346077602F466C
:10265000FFF706FFFFF762FE31680F607768083604
:10266000FFF75CFE0A490F60802731680F43094875
:102670000568002D01D140200743FFF711FF0549F0
:1026800000200860FFF78AFF00BD00002C1000202A
:102690003810002000100020002F80CE00B506D09A
:1026A000074805682D1D361F37602F4604E0054892
:1026B0000568361F37602F46FFF7D2FE00BD0000C9
:1026C000181000201C10002000B5FEF711FE00BD00
:1026D00000B5FEF70DFE7D1C3F78361F356000BD4E
:1026E00000B5FEF705FE30680028EFF3008001B466
:1026F000361D01BC80F3008805D05D462F65034F71
:1027000000F034F800E080CE00BD0000FEFFFFFFC7
:1027100000B5FEF7EDFD00F0D3FA00BDA4230008DC
:10272000C543415443482020361F3760374600B523
:1027300080B44F4680B45F463F6C80B46F465D46C0
:102740002F6435687768083601200543A84720BC08
:102750005C46256401B001B0361F3760002700BD1C
:102760007C240008C55448524F572020002F00B544
:1027700001D180CE00BD5D462D6CAD4620BC5C46CF
:10278000256420BCA94620BC80B42F463E1C80CEC8
:1027900080BC00BD9C240008C63F5448524F5720BF
:1027A00030680028EFF3008001B4361D01BC80F3CF
:1027B000008800B502D0FFF7D9FF00E080CE00BD51
:1027C0006C2300088641424F5254222000B500F08D
:1027D00097FC361F3760034FFEF7AEFD00F028FF71
:1027E00000BD0000E0260008BC210008C348455891
:1027F0005D461020A8637047EC270008C744454396
:10280000494D414C5D460A20A8637047982700084F
:10281000C342494E5D460220A86370471423000856
:10282000C4484F4C442020205D460448E96B0918F9
:10283000E9635D46ED6B2F7080CE7047FFFFFFFFB1
:102840009C210008C12320205D46AD6B361F3760F8
:102850002F4600B5FDF7D4FF70680928EFF300801C
:1028600001B43D46776831687160356001BC80F322
:10287000008800DDFF1D3037FFF7D6FF00BD0000E8
:1028800010280008C223532000B500BFFFF7DCFF6B
:1028900035683D43002DF9D100BD00002822000815
:1028A000C23C23205D4698355C46E56370470000D6
:1028B00084280008C2233E205F46FF6B5D469835A2
:1028C000ED1B37602F467047C4270008C3442E52C3
:1028D00000B580B437687068316871603060FDF7AA
:1028E000B9FEFFF7DFFFFFF7CFFF70680028EFF3B7
:1028F000008001B431687160361D01BC80F300882E
:1029000004D5361F37602D27FFF78EFFFFF7D4FF62
:1029100020BCED1B361F37602F46FFF7E5FCFFF7A5
:10292000B3FC00BD3C240008C2442E20361F376093
:10293000002700B5FFF7CCFFFFF7C8FC00BD000083
:1029400040220008C12E2020FD17361F37602F4679
:1029500000B5FFF7EBFF00BDCC280008C2552E20C4
:10296000361F3760002700B5FFF7E0FF00BD00000D
:1029700020270008C3552E52361F0021316000B5B4
:10298000FFF7A6FF00BD000098200008C22E5220CD
:1029900000B580B43168CF1720BC361F37602F4692
:1029A000FFF796FF00BD20205D46AD6B361F7168B6
:1029B000316077602F4600B5FDF772FE5F46BF6B52
:1029C0003568B16831607168B1607560FDF768FEA7
:1029D000FDF706FE5D466D6C6D1C03D05D46696CAF
:1029E000491C696400BD0000B4280008C73E4E556C
:1029F0004D424552083E37607760002700B500BF62
:102A0000FDF77AFD652A000835682D78361F376096
:102A10002F46FEF7F1F95D46AD6B361F37602F4646
:102A2000FEF74CFB002F01D0002701E001277F4279
:102A3000002F80CE01D002B000BD3168706801B4B3
:102A400002B40836FFF7B0FF20BC10BC0123ED1A1A
:102A50001B19083E336077602F460098401C009099
:102A6000D2D703B000BD20205D462F48686435688A
:102A70002D782D2D01D0002501E001256D4200B5F6
:102A800020B4002D04D001257F1B30682D1835603F
:102A9000012F03DA01B00027361D00BD083EB168E2
:102AA0003160002171600021B16000BFFFF7A2FF1B
:102AB000002F22D001257F1B30682D18356000BF04
:102AC0003068451E2D783A2DEFF3008001B4361F93
:102AD00037602F4601BC80F3008801D180CE0BE027
:102AE0002E2F04D15F460020786480CE04E001B030
:102AF0000027103600BD80CED8E780BC002FEFF352
:102B0000008001B47768083601BC80F3008801D0EA
:102B1000FDF77EFD5D466D6C002D01D5012702E0BD
:102B2000361F3760022700BDFFFFFFFF00B500BF63
:102B300035682D78242DEFF3008001B4361F3760FF
:102B40002F4601BC80F300880AD101273168CD1BD4
:102B500070683F1877602F46361DFFF749FE1BE06F
:102B6000232F0AD101273168CD1B70683F18776089
:102B70002F46361DFFF746FE0EE0252F0BD101270D
:102B80003168CD1B70683F185C460220A0637760F7
:102B90002F46361D00E080CE00BD000084200008D6
:102BA000C8494E54454745523F2020207D1C3F7860
:102BB000002FEFF3008001B4361F356001BC80F3B5
:102BC000008800B510D0083EB16831607760FEF72C
:102BD00021F95D46AD6B20B4FFF7A8FFFFF744FF76
:102BE00020BC5C46A56301E00027361D00BD000047
:102BF000EC290008C74E554D4245523F00B500BF75
:102C0000FEF7D8FC901000205D466D6B361F3760D4
:102C10002F46002F00D180CE00B50FD0361F376071
:102C20000827FFF71FFBFFF751FB361F3760082708
:102C3000FFF718FB7F1E5D466F6380CE00BD20202E
:102C4000002F01D1002501E001256D425C46246B77
:102C5000002C01D1002401E0012464422C4000B585
:102C600006D0FFF7D1FF7F1E361F3760024F02E00C
:102C7000361F3760002700BDFFFFFFFF3068387048
:102C80005F463F6B002F80CE00B502D0FFF7EAFA17
:102C900000E080CE00BD00008C290008822E22209A
:102CA000361F3760034F00B5FEF746FB00F0C0FC4F
:102CB00000BD00001027000828290008C2242E208B
:102CC0007D1C3F78361F356000B5FFF7DDFA00BD8B
:102CD0005C290008C641434345505420002F00B5ED
:102CE00001D1361D00BD5D46ED6A002D04D0361FB2
:102CF00037601127FFF7B6FA30683F18361F376084
:102D000077680021716000BFFDF7F6FBAB2D00086E
:102D1000FFF78CFA082F03D180CEFFF791FF3EE03A
:102D2000092F0CD1009F01980744361F20213160E4
:102D3000FFF7A4FF7F1C361F376001272FE00A2F03
:102D400001D100272BE00D2F0AD1009F01980744E5
:102D5000361F20213160FFF791FF02B000BD1EE059
:102D60000C2F0AD1009F01980744361F20213160A3
:102D7000FFF784FF02B000BD11E07F2F03D180CEAA
:102D8000FFF75EFF0BE0009D01980544361F37609A
:102D90002F46FFF773FF7F1C361F3760012700980F
:102DA000C019009080CEB3D703B05D46ED6A002D08
:102DB00004D0361F37601327FFF754FA00BD000018
:102DC00000B500BFFEF7B8FB941000205D466D6AA9
:102DD0005C46246A083E35607760274670470000ED
:102DE000BC2C0008C55155455259202000200949E6
:102DF00008605D466D6A083E35607760FF2700B564
:102E0000FFF76CFF5D462F625F460020B86280CE00
:102E100000BD00009410002074290008C6524546E9
:102E2000494C4C2007480568002D00B503D0361FDB
:102E30003760002704E0FFF7D9FF361F3760024FE5
:102E400000BD000094100020FFFFFFFFF42B0008DE
:102E5000C55041525345202000B580B480CEFFF7C5
:102E6000B5FF5D46AD6A7F1B30682D1810BC083E6B
:102E700037607560B5602746FDF76CFE80B4316839
:102E800070680F1A20BC002D01D1002501E001253A
:102E90006D427D1B5C46A16A4919A162361D00BDC9
:102EA00000B580B480CEFFF791FF5D46AD6A7C1B14
:102EB00030682D18009B083E34607560B7601F466F
:102EC000FDF734FE20BC083E3760B16871602F46C4
:102ED000FDF740FE80B4316870680F1A20BC002DE9
:102EE00001D1002401E0012464426419B1680C1B83
:102EF0005D46AC627168B160083600BDFC27000811
:102F0000C4574F524420202000B5FFF7C9FF0648A0
:102F10000568361F37602F46FDF7A0FF0248056899
:102F2000361F37602F4600BD1C10002000B5FFF78C
:102F30008BF9002F00D100BDFFF778F9202F80CE4C
:102F400008D180CEFFF772F9202F01D1002701E0D0
:102F500001277F4200BD2020002F00B501D001488D
:102F60003F1A00BD000000085D469835044804681B
:102F70002468A4006419083E346077602F467047C7
:102F800030100020083E002131607760002700B536
:102F9000FFF7EAFFFDF7A4FAC52F0008009D01988E
:102FA00005442D68AF4208D2009F01980744009D58
:102FB000019805442D6837602F460098001D009049
:102FC000ECD703B0002F01D001483F1800BD80F3BB
:102FD00000000008104805682D1D361F37602F4679
:102FE00000B5FFF7C1FF00BFFDF77AFA1530000802
:102FF0003D68361F37602F46FFF7AEFF009D0198F2
:1030000005442F6037683F1D361D0098001D009055
:10301000EED703B080CE00BD30100020202800087D
:10302000C5574F524453202000B5FFF73DF9FFF735
:10303000D1FF00BFFFF7A6FF361F3760FFF776FF0F
:10304000002F01D0002701E001277F4231680F40A7
:10305000EFF3008001B47768083601BC80F3008884
:1030600012D05D466D6B402D01DDFFF71DF9361F57
:103070003760FFF787FA3F1F3F68FFF76DFF316842
:103080000F6077680836D5E77768083600BD704668
:10309000401E02681268014B1A6000BD301000200B
:1030A0003068874201D1002701E001277F42376065
:1030B000024F00B5FFF774FB00BD0000EAFFFFFF01
:1030C000361F3760374602490F6080CE70470000D8
:1030D00020100020361F3760374607480568BD427C
:1030E00001D1002701E001277F42361F3760034FDF
:1030F00000B5FFF755FB00BD20100020EAFFFFFFE1
:1031000007480568002D01D0002501E001256D422A
:10311000083E35607760034F00B5FFF741FB00BD07
:1031200028100020F2FFFFFF04480568083E3560C4
:103130007760034F00B5FFF733FB00BD2810002078
:103140006DFEFFFFE42D000882444F2000B5FFF71D
:10315000D7FFFEF74FFB361F3760032700BD000087
:1031600034230008833F444F00B5FFF7C9FFFEF743
:103170004FFB361F3760032700BD00009C2C000862
:10318000844C4F4F5020202000B5FFF7B9FF361F69
:1031900037600327FFF784FFFEF748FB00BD000000
:1031A00080310008852B4C4F4F50202000B5FFF791
:1031B000A7FF361F37600327FFF772FFFEF744FBB8
:1031C00000BD0000D42C000885424547494E202010
:1031D00000B5FFF795FFFEF7B3FA00BD48310008D0
:1031E00085414741494E202000B5FFF789FFFEF792
:1031F000B1FA00BDFC24000885554E54494C2020EE
:1032000000B5FFF77DFFFEF7B1FA00BD20300008E2
:10321000855748494C45202000B5FFF771FFFEF760
:10322000BDFA30683760074600BD00001C2E00085C
:10323000865245504541542000B5FFF761FFFEF727
:1032400089FAFEF771FA00BD002F00088249462076
:1032500000B5FFF755FFFEF7A1FA00BD30320008B8
:10326000845448454E20202000B5FFF749FFFEF763
:103270005BFA00BD6427000884454C53452020209C
:1032800000B5FFF73DFFFEF77DFA3068376007466F
:10329000FEF74AFA00BD0000783200088752454325
:1032A0005552534505480568361F37602F4600B50F
:1032B000FDF786FEFEF740F800BD00008C100020F0
:1032C000C8310008844341534520202000B5FFF752
:1032D00017FF06480568361F37602F46FEF7C8FA05
:1032E000FFF7EEFE361F3760042700BD20100020D8
:1032F000A02B0008824F4620361F3760042700B5F8
:10330000FFF7CEFEFEF7C2FA361F3760052700BD75
:1033100064310008833F4F46361F3760042700B5ED
:10332000FFF7BEFEFEF7ECFA361F3760052700BD3B
:10333000F831000885454E444F462020361F37603F
:10334000052700B5FFF7ACFEFEF7ACFA361F376075
:10335000042700BD1032000887454E4443415345C1
:10336000361F3760042700B5FFF79AFEFEF7BCFA58
:1033700001490F6080CE00BD20100020361F37604D
:1033800037465D46AD69BD4201D3002701E0012704
:103390007F42361F3760024F00B5FFF701FA00BDCC
:1033A000FCFFFFFF002F01D0002701E001277F4233
:1033B000361F3760024F00B5FFF7F2F900BD00007D
:1033C000F3FFFFFF6032000888504F5354504F4EB8
:1033D00045202020361F3760202700B5FFF794FDD9
:1033E000FFF790F8361F3760FFF7DCFF0120C74278
:1033F00080CE04D100F060F8361F3760014FFDF732
:103400009BFF00BD38130008502E00088253222075
:1034100010480568002D00B507D0361F37600E4FE5
:10342000FDF78AFF00F004F913E0361F376022270A
:10343000FFF712FD5D469835361F37602F46FDF7C2
:103440000DFD5D4698356C1C2D78083E3460776024
:103450002F4600BD28100020D02600080C3400089C
:10346000824322200F480568002D00B507D0361F83
:1034700037600D4FFDF760FF00F0DAF810E0361FFF
:1034800037602227FFF7E8FC5D469835361F376026
:103490002F46FDF7E3FC5D469835361F37602F4613
:1034A00000BD000028100020C82600087C25000868
:1034B000874C49544552414C00B5FEF77BF900BD9D
:1034C000C4320008C443484152202020361F3760D0
:1034D000202700B5FFF718FD7F7800BDF432000803
:1034E000865B434841525D2000B5FFF709FEFFF7B8
:1034F000EDFFFFF7E1FF00BD58330008815B20209E
:10350000014900200860704728100020A02800080A
:10351000C15D202002490120404208607047000040
:1035200028100020C8330008C1272020361F37602C
:10353000202700B5FFF7E8FCFEF7E4FFFFF732FFB6
:1035400000BD000010350008835B275D00B5FFF764
:10355000EDFFFFF7B1FF00BD44280008895B434F32
:103560004D50494C455D202000B5FFF7DFFFFDF7CA
:10357000E3FE00BD9C32000881282020361F376002
:10358000292700B5FFF7C0FC80CE00BD5C240008F1
:10359000815C2020361F3760002700B5FFF7B4FCA0
:1035A00080CE00BD00B5306801B480B477680836BD
:1035B000361F37602027FFF7A7FC3D78002D1CD071
:1035C0007D1C3F78009CBC42EFF3008001B42F4685
:1035D00001BC80F300880ED1009D019C083E346040
:1035E00077602F46FDF7C8FA002F80CE02D020BCAE
:1035F00010BC00BD00E080CEDAE780CEFFF712FC01
:10360000002F80CED4D120BC10BC00BD34330008C4
:103610008228282000B5FFF75BF802292900000066
:10362000FFF7C0FF00BD00005C350008C2222C205F
:10363000361F3760222700B5FFF766FC3D786D1C0A
:10364000361F37602F46FEF7A9FF00BD00B520BC2E
:10365000E41D03218C4310B42D682F6080CE00BD83
:103660004C3200088249532000B5FFF75FFFBF6866
:1036700008480568002D07D0361F3760064FFDF754
:103680005BFEFEF7EDFE03E03068386077680836D1
:1036900000BD0000281000204C36000878350008D6
:1036A000844558495420202000B5FFF729FDFEF736
:1036B00097F800BDFC340008813B202000B5FFF7DF
:1036C0001FFDFFF707FDFEF78BF8FEF70BFFFFF777
:1036D00017FFFEF727FC00BD14330008C9494E54FC
:1036E000455250524554202000B500BFFFF746FE1A
:1036F000361F37602027FFF707FC3D78002D3FD0AD
:10370000FEF700FF002F00D180CE13D0002F01D490
:10371000002701E001277F421A4805683D4080CE1E
:1037200002D0FDF709FE04E03D4680CE01200543AE
:10373000A84724E0FFF762FA002F01D0361F376058
:10374000FFF730FE0F480568002D17D0012F03D179
:1037500080CEFEF72FF810E0022F08D1776831688D
:103760007160361DFEF726F8FEF724F805E0361FD7
:103770003760054FFEF7FAFF80CE00E080CEB5E758
:1037800080CE00BD28100020F3FFFFFF9035000819
:10379000C84556414C554154452020205D466D6A30
:1037A00000B520B45D462D6A20B45D46AD6ABD42C9
:1037B00001DB002701E001277F421048056820B4A3
:1037C0005D462F625F46306878620D480B4908609D
:1037D0005F460020B8620B4F361DFEF7A5FF20BCE8
:1037E00006490D6020BC5C46A56220BC5C46256293
:1037F00020BC5C466562FEF7B9FF00BD9410002056
:10380000FFFFFFFFE836000800B500BF002F01D121
:1038100080CE25E00120C74201D180CE20E00220E9
:10382000C74204D15F463F6DFFF74AFA18E00D200A
:10383000C7420AD180CEFEF76BFF0C697320756E0C
:10384000646566696E6564000AE0FEF761FF0B540B
:1038500068726F7720636F6465200000FFF774F86B
:1038600000BD000060340008C45155495420202098
:103870005D460020E8625D4601204042286300204A
:103880002F49086000B5FFF73BFE00BF5D46ED69BC
:10389000AD465D462D6B002D01D0FEF705FDFFF70F
:1038A000A5FA361F3760274FFEF73EFF002F24D1C1
:1038B00025480768002F01D0002701E001277F423B
:1038C0005D462D6B002D01D1002501E001256D42E3
:1038D0003D4080CE10D0FEF71BFF03206F6B000031
:1038E000FDF7F6F8002F00D180CE05D0FEF710FFCF
:1038F000012D0000FFF728F820E0FFF785FF5D4667
:10390000AD69361F37602F463E1C80CEFFF7F8FDAD
:10391000FEF7CAFCFFF75AFAFEF7B6FCFEF7C4FC46
:103920005D46AD6A6D1E361F37602F46FEF7DCFC24
:10393000FEF7EEFE015E0000FEF7F4FAA6E700BD1A
:1039400094100020E83600082810002000550008D8
:10395000B00F0008B8360008C9434F4C44434841F3
:10396000494E202000B500BFFDF7E6FD981000206D
:10397000C4340008C64154434F4C442000B5FEF700
:1039800061FDFEF7CBFC054805682F6003490F6019
:103990000027FEF765FDFEF763FD00BD98100020CF
:1039A0002C360008CD57414C4B434F4C44434841C3
:1039B000494E2020361F3760054F00B5002F05D037
:1039C0007D6801200543A8473F68F7E780CE00BD2A
:1039D0004C390008361F3760004F01E07C71000849
:1039E00000B500BF3D68002D0FD03D460C353C684A
:1039F0007B680C3E33607560B7602746FDF7A2F91F
:103A00003D68ED190C352F46ECE75F461837083E48
:103A10003760144971601027FDF794F95D46AD6970
:103A2000361F37602F463E1C80CE5D460E486862CA
:103A30005D46002028640C3E0C4931600C497160E1
:103A4000B7600827FDF77EF900200A490860FEF7F5
:103A5000D9FE094D09490D6009490D600020094949
:103A6000086000BDF8010008200C0020181000209C
:103A70001C02000894100020481000203010002084
:103A80002C10002034100020B0340008C52E4652FF
:103A90004545202000B5FEF707FC16480568164985
:103AA0004D1B083E356077600027FEF73FFFFEF7AD
:103AB0002FFE106279746573206672656520466C0E
:103AC00061736800FEF7F0FB03F052FB0B480568DA
:103AD0007F1B361F37600027FEF728FFFEF718FE12
:103AE0000E627974657320667265652052414D00DF
:103AF00000BD00001810002000F001081C1000207C
:103B0000A0360008C6434F4D4D495420002F00B544
:103B100000D1074F0120074306490F60083E742774
:103B20000549316005497160FEF774F900BD000078
:103B3000B00F00083C10002000F801081810002009
:103B400010360008C5454D5054592020083E0849FC
:103B500031607760742700B5FEF708F9083E054923
:103B600031607760044FFEF701F900F087F800BD7F
:103B700000F8010800C000080030010048350008C6
:103B8000C628434F4C44292000B5FFF723FF00F01F
:103B9000ADFF00F09DFF5D46AF6480CE00F098FF62
:103BA0005D46EF64083E74272749316027497160FC
:103BB000FEF730F9264805680120C54201D10024EE
:103BC00001E001246442002D01D1002501E001251E
:103BD0006D42254011D01F4805681F480468AC425B
:103BE00009D10C3E1949316019497160B7607427D9
:103BF000FDF7A8F801E0FFF7A9FFFEF723FC134843
:103C000005682D680120C54201D0FFF79FFFFFF72F
:103C1000D1FEFEF749FB01F029FFFFF73BFFFEF75E
:103C2000EDFAFEF741FBFEF73FFBFEF771FD0420C6
:103C3000206F6B005D46AD69361F37602F463E1C16
:103C400080CEFFF715FE00BD00F00108181000201F
:103C500000F801082802000874F801087439000807
:103C6000C4434F4C4420202000B500F007F800BDAD
:103C700028350008C65245424F4F542072B60549B8
:103C800001200D6805430D6003480449086000B534
:103C9000FEE700BD24100240CCCC00000030004004
:103CA000F0B54046494652465B460FB46946F03986
:103CB0008B460A1CF03A95460E46083E341F8C612E
:103CC0006846C861FDF774F96946F031F0318D46F8
:103CD0000FBC8046894692469B46F0BD1F253D405D
:103CE0000124AC407F09BF00361F346070470000DC
:103CF000443B0008C5454E494E5420200F2F00B5C7
:103D00000BD9103FFFF7EAFF05483F1805483F1859
:103D1000306838607768083600BD80CE00BD00008E
:103D200000E000E000010000F43C0008C6444953F4
:103D3000494E54200F2F00B50BD9103FFFF7CEFF8F
:103D400005483F1805483F183068386077680836DE
:103D500000BD80CE00BD000000E000E0800100005A
:103D6000743C0008C92F4150504652414D45202017
:103D700000B500BFFDF7A3FB20000000643600087B
:103D8000C64558412E52302000B500BFFFF7FFFF57
:103D900000000000803D0008C64558412E523120E9
:103DA00000B500BFFFF7FFFF04000000983D0008CA
:103DB000C64558412E52322000B500BFFFF7FFFF25
:103DC00008000000B03D0008C64558412E5233207F
:103DD00000B500BFFFF7FFFF0C00000058390008D6
:103DE000C74558412E52313200B500BFFFF7FFFFE3
:103DF00010000000E03D0008C74558412E52313404
:103E000000B500BFFFF7FFFF14000000C83D000829
:103E1000C64558412E50432000B500BFFFF7FFFFB5
:103E200018000000F83D0008C74558412E50535275
:103E300000B500BFFFF7FFFF1C000000043B0008B7
:103E4000CA2F4D41494E4652414D452000B500BF55
:103E5000FDF735FB24000000103E0008C645584D14
:103E60002E52342000B500BFFFF7FFFF0000000016
:103E70005C3E0008C645584D2E52352000B500BFA7
:103E8000FFF7FFFF04000000743E0008C645584DD0
:103E90002E52362000B500BFFFF7FFFF08000000DC
:103EA0008C3E0008C645584D2E52372000B500BF45
:103EB000FFF7FFFF0C000000A43E0008C645584D68
:103EC0002E52382000B500BFFFF7FFFF10000000A2
:103ED000BC3E0008C645584D2E52392000B500BFE3
:103EE000FFF7FFFF14000000283E0008C745584DAB
:103EF0002E52313000B500BFFFF7FFFF1800000061
:103F0000EC3E0008C745584D2E52313100B500BF78
:103F1000FFF7FFFF1C00000044290008CA45584D68
:103F20002E4558435245542000B500BFFFF7FFFF10
:103F300020000000E0310008C72F4558444154419B
:103F400000B500BFFDF7BBFA140000001C3F0008DD
:103F5000CA4558442E523133464C542000B500BF58
:103F6000FFF7FFFF00000000A4310008CB455844D4
:103F70002E5231334D41494E00B500BFFFF7FFFFD0
:103F8000040000008C3A0008CE4558442E523133CC
:103F900050524F434553532000B500BFFFF7FFFF7A
:103FA00008000000E0340008CC4558442E5231335C
:103FB000535441544520202000B500BFFFF7FFFFB8
:103FC0000C000000503F0008CA4558442E4C524D8A
:103FD00041494E2000B500BFFFF7FFFF1000000071
:103FE000D43E0008C64558444154412000B500BFA6
:103FF000FDF765FA4C060020164BEFF30880586079
:10400000EFF30981996072461A610420024201D1DE
:10401000586800E0986818604046494652465B463A
:104020000FB5F0B40B4B6846D860F8B06846F03076
:1040300083460646083E341F84616946C161FCF729
:10404000B7FF78B0F0BC0FBC8046894692469B46CD
:1040500000BD00004C060020883F0008C52E4954D2
:10406000454D20203D68361F37602F4600B500F0D3
:104070009FFDFEF72BF93F1D00BD0000A43900088D
:10408000C62E4954454D5320361F3760002700B5D2
:10409000FCF732FAA7400008FFF7E4FF0098401C45
:1040A0000090F9D703B000BD403E0008C841505011
:1040B0004954454D5320202002480568361F37607B
:1040C0002F4670474C060020383F0008C94D414933
:1040D0004E4954454D53202002480568361F37602D
:1040E0002F46704758060020603C0008C6415050DB
:1040F0005253502000B5FFF7DFFF203700BD00000E
:10410000EC400008C64150505053502000B5FFF716
:10411000E3FFBF6800BD0000CC400008C54150501F
:104120005550202000B5FFF7D7FFFF6900BD000004
:1041300004410008C6415050544F532000B5FFF7CA
:10414000CBFFFF6800BD00001C410008C541505076
:104150005043202000B5FFF7AFFFBF6900BD00004E
:1041600034410008C92E464C544652414D4520204A
:1041700000B5FFF7A1FFFEF797F8FEF7C9FA113D6A
:104180003D3D20526567697374657273203D3D3D06
:10419000FEF78AF8FEF7BCFA06505352203D200085
:1041A000FD69361F37602F4600F002FDFEF77CF8F0
:1041B000FEF7AEFA06523020203D2000083E376060
:1041C00077600427FFF760FF80CEFFF785FFFEF7DB
:1041D0006BF8FEF79DFA06523420203D20000000C7
:1041E000361F37600427FFF74FFFFEF75DF8FEF735
:1041F0008FFA06523820203D20000000361F37601D
:104200000427FFF741FF80CEFFF756FFFEF74CF87B
:10421000FEF77EFA06523132203D20003D46103531
:10422000361F37602F46FFF71DFF3768203700F035
:10423000BFFCFEF74BF81437361F37600227FFF735
:1042400023FF80CE00BD00005C400008C54E414DFC
:10425000453F2020FD1C03218D43AF4200B501D016
:10426000002700BD7D1C3F789F243C40103E8121EB
:1042700031607460B760F560A027FCF7D9F8002FB3
:1042800080CE02D10027361D00BD1F2007403068B8
:104290003F18306837600746FCF72EF9D342000814
:1042A000009D019805442D780C3E212131607560F8
:1042B000B7607F27FCF7BCF8002F80CE04D103B095
:1042C000361F3760002700BD0098401C0090E7D7DC
:1042D00003B0361F3760014F00BD0000FFFFFFFF36
:1042E000C83F0008C649503E4E464120BF1E00B59B
:1042F000361F3760FFF7AEFF002F80CE01D17F1E43
:10430000F6E700BD6C3F0008CD434845434B2D41C7
:104310004C49474E45442020FD1C03218D43AF42AC
:1043200000B50CD0FEF7F4F90D284D6973616C6986
:10433000676E656429200000FF1C03218F4300BDC8
:104340004C410008C73F434C4950333230683D1A56
:10435000802D00B510D937688037FDF7A5FFFEF72F
:10436000D7F913436C697070656420746F20333221
:10437000206974656D73000000BD000044430008AF
:10438000C82E52534641554C5420202000B5FDF70D
:104390008BFFFFF7AFFEFDF787FFFEF7B9F9065277
:1043A0005350203D20000000361F376000F000FC15
:1043B000FDF78CFFFFF7B0FFFFF7B4FEFF69FEF7D4
:1043C000A7F90720205230203D200000361F37601B
:1043D00000F0EEFBFDF77AFFFFF79EFF3F1FFDF7B2
:1043E00063FFFEF795F9192D2D2D20526574757216
:1043F0006E20737461636B2068696768202D2D2DB2
:10440000FFF7A4FFFCF778F869440008FDF74CFFBC
:10441000009D01980544361F37602F4600F0C8FB09
:10442000FDF754FF009D019805442D68083E356056
:1044300077602F4600F0BCFBFDF748FF0C3E1449A7
:1044400031607760B760134FFBF7F2FF002F80CE2B
:1044500004D0FFF74BFFFEF795F800E080CE009800
:10446000001F0090D2D703B0FDF71EFFFEF750F9F2
:10447000192D2D2D2052657475726E207374616331
:104480006B206C6F77202D2D2D20000000BD0000CB
:104490003402000800C0000880430008C82E5053B2
:1044A0004641554C5420202000B5FDF7FDFEFFF796
:1044B0002DFEFDF7F9FEFEF72BF906505350203D77
:1044C00020000000361F376000F072FBFDF7FEFE93
:1044D000FFF722FFFFF726FEBF69FEF719F9072055
:1044E000205330203D200000361F376000F060FB75
:1044F000FDF7ECFEFFF710FF3D1D3068854212D23C
:1045000077680836FDF7D0FEFEF702F916446174AD
:104510006120737461636B20756E646572666C6F85
:104520007765640000BD3D1D306885420FD1776816
:104530000836FDF7B9FEFEF7EBF810446174612010
:10454000737461636B20656D7074790000BD3068B1
:104550003D1AF02D11D977680836FDF7A5FEFEF754
:10456000D7F8154461746120737461636B206F76B2
:104570006572666C6F77656400BDFDF795FEFEF7AA
:10458000C7F8172D2D2D2044617461207374616369
:104590006B2068696768202D2D2D000030688742E8
:1045A00021D03F1FFFF7D2FEFBF79AFFE545000839
:1045B000FDF77AFE009D01980544361F37602F46AF
:1045C00000F0F6FAFDF782FE009D019805442D6883
:1045D000361F37602F4600F0EBFA0098001F00905E
:1045E000E6D703B001E077680836FDF75DFEFEF719
:1045F0008FF8172D2D2D2044617461207374616331
:104600006B206C6F77202D2D2D200000FDF74CFEC8
:10461000FEF77EF80972544F532F523720200000C6
:10462000FFF78CFD00F0C4FA00BD0000043F000855
:10463000C953484F574641554C54202000B500F00F
:1046400047FA5D46EF645D46AF6480CE00F09AF9AC
:10465000FEF7D8F8083E354931607760002700BF83
:10466000FBF73EFF734600080098401C0090FBD704
:1046700003B0083E0521316077600027FBF730FF6B
:1046800099460008361F37600527FDF7EBFD0098B7
:10469000401C0090F6D703B001F076FFFDF704FE52
:1046A000FDF702FEFEF734F80A4578636570746919
:1046B0006F6E2000EFF30585361F37602F46FEF73B
:1046C00043F9FEF725F8036174200000FFF742FD6F
:1046D00000F06EFAFFF74CFDFFF758FEFFF7E4FE1F
:1046E000FDF7E2FDFEF714F81552657374617274FC
:1046F000696E672073797374656D202E2E2E00000D
:10470000083E0A4931607760002700BFFBF7E8FEEA
:104710001F4700080098401C0090FBD703B0FFF72C
:10472000ADFA361F3760002700BD000010270000DB
:10473000164BEFF308805860EFF3098199607246D9
:104740001A610420024201D1586800E0986818609C
:104750004046494652465B460FB5F0B40B4B68469F
:10476000D860F8B06846F03083460646083E341FED
:1047700084616946C161FFF761FF78B0F0BC0FBC8E
:104780008046894692469B4600BD00004C060020AC
:10479000164BEFF308805860EFF309819960724679
:1047A0001A610420024201D1586800E0986818603C
:1047B0004046494652465B460FB5F0B40B4B68463F
:1047C000D860F8B06846F03083460646083E341F8D
:1047D00084616946C161FFF731FF78B0F0BC0FBC5E
:1047E0008046894692469B4600BD00004C0600204C
:1047F00090370008CA53454C494F2D53455231203C
:104800001A4D2C463034103E032131600021716076
:10481000B560F760274600B5FDF7A6F8144879693A
:10482000014379611248B96A8143B9621148B96993
:104830000143B9610F48F9688143F9600E4801B43A
:10484000009F3F1C083E0D4931600D497160FDF726
:104850008BF820BC24350C3E0A4931600A4971604E
:10486000B7602F46FDF780F800BD00000010024041
:1048700000000200004000000000004800003C0072
:1048800000002800F00F000010010000A83F000801
:10489000C9285345524B45593F292020FF69202004
:1048A0000740704708430008C8285345524B4559F4
:1048B0002920202000B500BFFD6920200540002DE3
:1048C00002D1FDF727F8F7E77F6AFF20074000BD18
:1048D00090480008C928534552454D495429202085
:1048E00000B500BFFD6980200540002D02D1FDF715
:1048F00011F8F7E73068B8627768083600BD000045
:10490000D4480008C92853455254595045292020FD
:10491000706831684518706877600746356000B583
:10492000FBF7EAFD45490008009D019805442D78F4
:10493000083E35607760FFF7D3FF0098401C009079
:10494000F2D703B080CE00BDE4420008C72853452B
:1049500052435229083E0D213160776000B5FFF7C0
:10496000BFFF361F0A213160FFF7BAFF00BD00000C
:10497000643D0008CD2B4641554C54434F4E534F98
:104980004C45202070470000DC360008CA28494EFC
:1049900049542D534552292000203860002078606A
:1049A0000020B8603068F8600C2038600D20386056
:1049B00077680836704700008C490008C9494E499D
:1049C000542D53455231202000B5FFF719FF083E02
:1049D000034931607760034FFFF7DEFF00BD000041
:1049E000A101000000380140E43F0008C8534552CF
:1049F0004B45593F31202020361F3760024F00B50C
:104A0000FFF74CFF00BD0000003801402C3D0008BE
:104A1000C75345524B455931361F3760024F00B5D9
:104A2000FFF748FF00BD000000380140EC490008D6
:104A3000C8534552454D495431202020361F376018
:104A4000024F00B5FFF74CFF00BD000000380140E9
:104A5000304A0008C853455254595045312020204F
:104A6000361F3760024F00B5FFF752FF00BD000050
:104A700000380140AC400008C65345524352312033
:104A8000361F3760024F00B5FFF764FF00BD00001E
:104A900000380140544A0008C8434F4E534F4C451C
:104AA0003120202000B500BFFCF709FDB04A000806
:104AB000184A0008F84900083C4A0008604A000803
:104AC000804A0008104A0008C7434F4E534F4C45D8
:104AD00000B500BFFCF7F3FCB04A00080449000829
:104AE000C8494E49542D53455220202000B5FFF7A8
:104AF0006BFF00BD80400008C62E4153434949204A
:104B00007F2007400C3E202131607760B7607F270F
:104B100000B5FBF78DFC002F80CE00D12E27FDF7CE
:104B2000A1FB00BD4C420008C52E4259544520202F
:104B30005D46AD6B00B520B4FDF75AFE361F3760F9
:104B40000027FDF7AFFEFDF77FFEFDF77DFEFDF7C9
:104B5000B3FEFDF799FB20BC5C46A56300BD0000D9
:104B6000284B0008C52E574F524420205D46AD6BA0
:104B700000B520B4FDF73CFE361F37600027FDF777
:104B800091FEFDF761FEFDF75FFEFDF75DFEFDF7AF
:104B90005BFEFDF791FEFDF777FB20BC5C46A5634D
:104BA00000BD0000F84A0008C62E44574F5244206A
:104BB0005D46AD6B00B520B4FDF71AFE361F3760B9
:104BC0000027FDF76FFEFDF73FFEFDF73DFEFDF709
:104BD0003BFEFDF739FE361F37603A27FDF724FE0E
:104BE000FDF732FEFDF730FEFDF72EFEFDF72CFE41
:104BF000FDF762FEFDF748FB20BC5C46A56300BDE7
:104C000074490008C444554D502020205D46AD6BCA
:104C1000361F71683160756000B5FDF7E9FD3068D9
:104C20003F18306837600746FBF766FCD94C000830
:104C3000FDF73AFB009D01980544361F37602F466B
:104C4000FFF7B6FF009D019805442C461034083E3E
:104C5000346077602F4600BFFBF742FC814C0008B0
:104C6000FDF734FB009D019805442D78361F376011
:104C70002F46FFF75DFF0098401C0090F0D703B06F
:104C8000361F37600227FDF72FFB009D0198054472
:104C90002C461034083E346077602F46FBF720FC2A
:104CA000C14C0008009D019805442D78361F3760DF
:104CB0002F46FFF725FF0098401C0090F2D703B065
:104CC000FDF7C2FA002F80CE01D002B000BD0098DF
:104CD00010300090ACD703B05D46AF6380CEFDF7D7
:104CE000E3FA00BD68380008C55044554D502020F7
:104CF0005D46AD6B361F71683160756000B5FDF7BC
:104D000077FD3068054603218D437F1937602F46B4
:104D1000FBF7F2FB814D0008FDF7C6FA009D0198F4
:104D20000544361F37602F46FFF742FF009D01986C
:104D300005442C461034083E346077602F4600BF8F
:104D4000FBF7CEFB694D0008FDF7C0FA009D019806
:104D500005442D68361F37602F46FFF729FF00985E
:104D6000001D0090F0D703B0FDF76EFA002F80CE43
:104D700001D002B000BD009810300090CCD703B035
:104D80005D46AF6380CEFDF78FFA00BDA8480008EE
:104D9000C22E532000B5FDF787FAFDF7B9FC032DAD
:104DA0002D200000FBF794FE002F00D180CE19D0FB
:104DB0007F1E361F00213160FBF792FBE54D000896
:104DC000009D01980544361F37602F46BF00F759F4
:104DD000361F37600027FDF7A9FD0098401E0090A0
:104DE000EED703B000BD0000A84B0008C450494FE7
:104DF0003A20202000B5FCF739FB31688D020B48C2
:104E00002D18361F37602F46FDF72AFB0125BD40C0
:104E1000361F37602F46FDF723FB31684D013D43B8
:104E20002F46361DFDF71CFB00BD000000000048AA
:104E3000BC490008C250412000B500BFFCF73FFB51
:104E400000000000344E0008C250422000B500BFF0
:104E5000FCF735FB01000000484E0008C25043201B
:104E600000B500BFFCF72BFB020000005C4E000801
:104E7000C250442000B500BFFCF721FB0300000036
:104E8000704E0008C250452000B500BFFCF717FB6C
:104E900004000000844E0008C250462000B500BF48
:104EA000FCF70DFB05000000784A0008C653455486
:104EB00050494E203D687F682F8380CE70470000A8
:104EC000AC4E0008C6434C5250494E203D687F68A6
:104ED0006F8380CE70470000F4470008C6474554F2
:104EE00050494E203D687F682D693D40002D01D11D
:104EF000002701E001277F42012007407047202062
:104F000003200740BD003D432F012F433D023D4399
:104F10002F042F43704720200F2007407F000325D8
:104F2000BD402F467047202030683760074600B5E7
:104F3000FFF7E6FF306837600746FFF7EDFF35689B
:104F40003D40356000BD2020BD680F200540361F64
:104F50007168316077602F4600B5FFF7E5FF75682F
:104F60002D683168716037602F4600BD984E00088B
:104F7000C9495350494E4D4F4445202000B5FFF7D5
:104F8000E3FF3F1CFCF7F0FC00BD20200F20074092
:104F90003D013D432F022F433D043D432F467047C3
:104FA00007253D40AD000F24AC40082007407F0896
:104FB000361F34607047202030683760074600B5E0
:104FC000FFF7E4FF306837600746FFF7E9FF80B47A
:104FD000376871680F4020BC77602F4600BD000025
:104FE000704F0008C9494E5055544D4F444520203C
:104FF00000B500BFFCF763FA00000000C44E0008D3
:10500000CA4F55545055544D4F44452000B500BF2C
:10501000FCF755FA0100000064410008C641464D06
:105020004F44452000B500BFFCF749FA02000000DC
:10503000984A0008CA414E414C4F474D4F444520C5
:1050400000B500BFFCF73BFA03000000904D0008DC
:10505000C74953494E505554361F0021316000B5A1
:10506000FFF78CFF00BD0000E04A0008C849534F1D
:105070005554505554202020361F0121316000B571
:10508000FFF77CFF00BD0000644B0008CA4953468F
:10509000554E4354494F4E2000B580B4009F361FF3
:1050A00002213160FFF76AFF009DAD680F200540C7
:1050B000361F37602F46FFF77FFF20BC2D68203555
:1050C000ED192F46FCF750FC00BD00006C500008A5
:1050D000C84953414E414C4F47202020361F0321E1
:1050E000316000B5FFF74AFF00BD000050500008D6
:1050F000C7495350494E4F4430680028EFF30080B1
:1051000001B4361D01BC80F3008800B506D03D68AF
:105110007F6869683943696080CE05E03D687F68D3
:105120006968B943696080CE00BD0000E44F0008A3
:10513000C9495350494E50555044202000B5FFF7FF
:1051400003FF0C37FCF710FC00BD00001C500008EA
:10515000C94E4F5450554C4C45442020361F002119
:10516000316000B5FFF7EAFF00BD0000044C000805
:10517000C850554C4C45445550202020361F012125
:10518000316000B5FFF7DAFF00BD0000C84A000833
:10519000CA50554C4C4544444F574E20361F0221AF
:1051A000316000B5FFF7CAFF00BD00008C50000859
:1051B000CA495350494E53504545442000B5FFF766
:1051C000C3FE0837FCF7D0FB00BD0000EC4D000823
:1051D000C84C4F57535045454420202000B500BFD0
:1051E000FCF76DF90000000070510008CB4D4544FC
:1051F00049554D535045454400B500BFFCF75FF994
:1052000001000000D0500008C948494748535045A4
:105210004544202000B500BFFCF751F90300000011
:10522000E84C0008C94C45444143544956452020A8
:1052300000B500BFFCF780F99C100020B0510008B9
:10524000C73C5449434B533E00B500BFFCF774F9CB
:10525000A010002000500008C55449434B532020A3
:1052600002480568361F37602F467047A01000209F
:105270004C490008C34C445500B500BFFCF71FF96A
:10528000845200080008004840000000460000006A
:1052900074520008C34C445200B500BFFCF70FF92C
:1052A000A452000800080048000200004900000065
:1052B00094520008C34C444400B500BFFCF7FFF80B
:1052C000C4520008000800488000000047000000A9
:1052D000B4520008C34C444C00B500BFFCF7EFF8D3
:1052E000E4520008000800480001000048000000E7
:1052F00030460008C95359535449434B4552202066
:1053000023490868401C086022480568002D00B544
:105310003DD000BF1E4805681F480540002DEFF333
:10532000008001B4361F37602F4601BC80F300882F
:1053300008D11A4FFFF7CAFD361F3760184FFFF725
:10534000B9FD24E01748874208D1154FFFF7BEFD8D
:10535000361F3760144FFFF7ADFD18E01348874242
:1053600008D1114FFFF7B2FD361F3760104FFFF71E
:10537000A1FD0CE00F48874208D10D4FFFF7A6FDB5
:10538000361F3760054FFFF795FD00E080CE00BD6A
:10539000A01000209C100020FF070000E45200082D
:1053A0008452000800020000A4520008000400001B
:1053B000C452000800060000F0B540464946524677
:1053C0005B460FB46946F0398B460A1CF03A9546A5
:1053D0000E46083E341F8C616846C861FFF790FF97
:1053E0006946F031F0318D460FBC804689469246C1
:1053F0009B46F0BD361F376000B5FFF73DFEFFF757
:1054000059FD00BD803B0008CB53544152542D43FD
:105410004C4F434B361F37600E4F00B5FFF7EAFF86
:10542000361F37600C4FFFF7E5FF361F37600B4F15
:10543000FFF7E0FF361F3760094FFFF7DBFF094D2D
:10544000094868610320286108496C18FF20207012
:1054500062B600BD84520008A4520008C45200087D
:10546000E452000800E000E06F170000230D000088
:10547000DC4E0008CA53544F502D434C4F434B2031
:10548000024901200D6885430D60704710E000E07F
:1054900008520008C54C4154455220200248056876
:1054A000ED192F4670470000A0100020745400082A
:1054B000C954494D45444F55543F20200448056880
:1054C0007F1B002F01D4002701E001277F42704796
:1054D000A0100020D4520008C24D53200748056890
:1054E000ED192F4600B500BFFCF714FA0348056814
:1054F0007D1B002DF8D580CE00BD01BCA010002082
:10550000EC5700081454000840520008C42F5443BC
:105510004220202000B500BFFBF7D1FF180000009B
:10552000F4520008C85443422E4C494E4B202020D0
:1055300000B500BFFFF7FFFF000000003450000877
:10554000C75443422E53535000B500BFFFF7FFFF2F
:105550000400000008540008CA5443422E5354412A
:105560005455532000B500BFFFF7FFFF08000000AF
:1055700024550008C85443422E4D53524320202046
:1055800000B500BFFFF7FFFF0C00000074550008D6
:10559000C85443422E4D45534720202000B500BF3C
:1055A000FFF7FFFF10000000B0540008C954434249
:1055B0002E4556454E54202000B500BFFFF7FFFF93
:1055C0001400000094540008C44D41494E2020208E
:1055D00000B500BFFBF773FF100F002000000000B4
:1055E000D8540008C7285041555345294846C1B5ED
:1055F000684659464860096888680028FBD08B4691
:1056000048688546C1BC814601BC8646704700009B
:105610000C550008864D554C54493F2000B500BF3D
:10562000FCF73BF8A410002058520008C653494E1E
:10563000474C45200348044908600020034908609E
:1056400070470000B10F00080C100020A4100020CB
:1056500030510008C54D554C544920200348044999
:10566000086004480449086070470000ED550008D0
:105670000C100020FFFFFFFFA41000202C56000894
:10568000C6535441545553205D46AD6801218D43A6
:10569000361F37602F46704780560008C752455363
:1056A000544152540120B9680143B96080CE70471B
:1056B00090550008C448414C542020200120B9686E
:1056C0008143B96080CE704750510008C453544F95
:1056D000502020205D462D1C361F37602F4600B518
:1056E000FFF7ECFFFCF716F900BD000002CE012326
:1056F00019436A463846F0388546F8610020B8609C
:1057000002B401B43946091E083902B401B4091FB4
:10571000B96168467860954680CE70475D462D68D1
:105720003D605D462F6080CE704720205D462D1C79
:10573000361F37602F4600B53D683068854208D077
:105740003F685D462D1CBD4202D17768083600BD1A
:10575000F2E735682D683D607768083600BD0000C7
:10576000C8550008C8494E49544941544520202095
:10577000361F71683160776000B5FFF7B7FF361FDD
:105780003760FFF7CBFF0120B86080CEFCF7C2F88E
:1057900000BD0000AC550008C95445524D494E416A
:1057A0005445202000B5FFF7C1FFFCF7B3F800BD5A
:1057B00014560008CA494E49542D4D554C544920A1
:1057C00000B5FFF737FF083E0649316077601827BC
:1057D000FBF768FB034D2D60012003490860FFF7CC
:1057E0003DFF00BD100F0020180F0020000000003A
:1057F000C057000840550008C34849535D462D1C5A
:105800007F1B30683F18361D70470000B4560008F3
:10581000C953454D4150484F52452020361F3760EF
:10582000082700B5FBF794FE0B4805680C3E0021E5
:10583000316000217160B7602F46FBF7C1FB3D4628
:1058400080CE01200543A8473068386070687860D2
:10585000B7680C3600BD0000381000209C560008C8
:10586000C65349474E414C2000B5FCF769F83868EB
:10587000401C38600020786080CEFCF76BF800BDDB
:1058800060580008C75245515545535400B500BFF4
:10589000FCF756F83D68002D04D1FCF75BF8FCF7E7
:1058A00039F8F5E73868401E38605D462D1C7D608C
:1058B00080CEFCF74FF800BD58550008CA5441533C
:1058C0004B2D434841494E2000B500BFFBF734FE45
:1058D000A8100020EC510008C45441534B20202054
:1058E00000B5FCF763FD0C4805680C482D18083E10
:1058F000356077600A4FFCF74BFDFBF7DBFDFCF7EB
:105900000DFD08480568361F37602F46FCF7A8FDD7
:1059100004490F6080CE00BD1C100020F001000083
:10592000E0020000A810002084580008C65354412B
:1059300052543A2000B520BC361F3560FFF718FFDF
:1059400000BD0000B4570008C52E5441534B202021
:10595000361F3760124F00B53F68002F0ED03D1F35
:105960002D683068854208D10C3F361DFBF73CFBA3
:10597000FCF708FEFCF7AAFC00BDEDE780CEFFF7C0
:1059800017F9FCF7C5FE15206973206E6F74206946
:105990006E205441534B20636861696E00BD000066
:1059A000A8100020D0510008C62E5441534B53205C
:1059B000361F3760094F00B53F68002F0BD03D46BA
:1059C0000C3D361F37602F46FBF70EFBFCF7DAFD68
:1059D000FCF77CFCF0E780CE00BD0000A8100020A2
:1059E0009C440008C82E52554E4E494E4720202058
:1059F000361F3760064F00B5FCF756FC361F376080
:105A0000FFF7A6FF3F6802488742F5D180CE00BD70
:105A1000100F00201276372E3330205B6275696CD0
:105A20006420303238305D153232204A616E2032C7
:105A30003032332C2031323A31333A353320202082
:105A400000B5FCF731FCFCF763FE1C2A2A2A2A2A3F
:105A50002A2A2A2A2A2A2A2A2A2A2A2A2A2A2A2AA6
:105A60002A2A2A2A2A2A2A0000BD202000B5FFF768
:105A7000E7FFFCF719FCFCF74BFE1C4D5045204698
:105A80006F727468204C69746520666F722053547D
:105A90004D33324630373200FCF706FC361F376094
:105AA000154FFDF70DF9FCF711FC361F3760134F4A
:105AB000FDF706F9FCF7F8FBFCF72AFE32436F709E
:105AC0007972696768742028432920323031342084
:105AD0004D6963726F50726F636573736F722045A7
:105AE0006E67696E656572696E67204C74642E001E
:105AF000FFF7A6FF00BD0000145A0008275A00084F
:105B000010580008CA524550524F472E494D472061
:105B100000B500BFFBF7D3FC1C5B0008FC070020AE
:105B20004409002000000000006CDC0200000200BC
:105B3000000800003B1C83CE00D17047021C0A43C2
:105B40001A430324144006D10A680260091D001D8F
:105B50001B1FF9D170470A780270491C401C5B1E5C
:105B6000F9D1704702CE0124E40773465B1E1A6820
:105B70000919781A07B480CE7046001D004700004E
:105B800002CEB942EFD180CE01217046884302682F
:105B90001047361F37607046401E076800BD000082
:105BA00072B670473A4603CE0027121A091A91427C
:105BB00000D2FF437047000001CE3168202400224C
:105BC0004918404113465341C01B5B4101D0491C59
:105BD00000E0C019641EF3D10F46306070472020EA
:105BE000361F0021316000B5FFF7E6FF361D00BD0E
:105BF0000038014007480568002D03D005480568B6
:105C000005490D60044805680C2028600D202860B7
:105C10007047000008000020D400002007480568F5
:105C2000361F37602F4600BFFD6980200540FBD03E
:105C30003068B8627768083670470000D4000020EA
:105C400004480568ED6920200540361F37602F465F
:105C500070470000D40000200A480568361F3760EE
:105C60002F4600BFFD6920200540FBD07F6AFF2042
:105C7000074000BF00BF00BF00BF00BF00BF00BFA4
:105C800000BF7047D400002030683F18306837608C
:105C9000074600B5FFF774FF9D010020009D0198A5
:105CA00005442D78361F37602F46FFF7B7FF009861
:105CB000401C0090F2D703B000BD2020361F376093
:105CC0000D2700B5FFF7AAFF361F37600A27FFF739
:105CD000A5FF00BD07480568083E35607760064FA0
:105CE00000B5FFF77DFF00BF7F1E002FFCD180CEE7
:105CF00000BD01BC0C00002020A10700074805687A
:105D0000083E35607760064F00B5FFF769FF00BFBA
:105D10007F1E002FFCD180CE00BD01BC0C000020F6
:105D20008813000000B500BFFFF7E8FF7F1E002FBB
:105D3000FAD180CE00BD202000B5FFF731FF054924
:105D400001200D6805430D6003480449086000BF49
:105D5000FEE700BD24100240CCCC00000030004023
:105D600000B500BFFFF715FF200A002000B500BFF7
:105D7000FFF70FFF240A002000B500BFFFF709FF5F
:105D8000280A002000B500BFFFF703FF2C0A0020FF
:105D900000B500BFFFF7FDFE300A002000B500BFD0
:105DA000FFF74EFF002F80CE03D0FFF755FF80CEC8
:105DB000F6E700BD361F3760062700B5FFF72EFF58
:105DC00000BD2020361F3760152700B5FFF726FFDE
:105DD00000BD2020361F3760182700B5FFF71EFFD3
:105DE000024901204042086000BD0000300A002046
:105DF000361F3760074F00B5FFF722FF002F80CE18
:105E000003D0FFF729FF361D00BD7F1E002FF3D101
:105E1000014F00BD00004000FFFFFFFF083E0021D2
:105E2000316077600C4F00B5FFF7E2FF31680F700B
:105E300070683F18FF20074035686D1C0748854291
:105E4000EFF3008001B477602F46361D01BC80F36C
:105E50000088E9D380CE00BD400A0020C00A00209F
:105E600000B5FFF7B7FFFFF7B5FF00BD00B5FFF7BF
:105E700095FF07490868401C086005480568054803
:105E8000854202DDFFF7ECFF01E0FFF79BFF00BD5D
:105E90002C0A00200001000007480568083E074959
:105EA000316077602F4600B500F0BCF90249086800
:105EB0008030086000BD0000240A0020400A002055
:105EC00000B5FFF795FFFFF793FF30683F18FF2FEE
:105ED00080CE05D0FFF7CAFFFFF77CFF80CE00BD64
:105EE00018480568FF200540BD4280CE02D0FFF76C
:105EF000BDFF00BDFFF792FFFFF77AFF30688742D2
:105F0000EFF3008001B47768083601BC80F30088A5
:105F100002D0FFF7ABFF00BD0A4805680A480468D5
:105F2000AC4202DAFFF79CFF00BDFFF7B5FFFFF7B9
:105F300041FF04490868401C0860044900200860CB
:105F400000BD0000200A0020280A00202C0A0020A2
:105F5000361F37600A4F00B5FFF772FE002F01D0E1
:105F6000002701E001277F423068074080CE03D040
:105F7000FFF7B0FE7F1EEFE780CEFFF761FE00BDAA
:105F8000A086010000B5FFF7E3FF002F80CE03D10C
:105F9000024901204042086000BD0000300A002094
:105FA0002A49002008602A490020086000B5FFF750
:105FB000F5FEFF0927490F60306827490860012076
:105FC000264908601527361DFFF728FEFFF7C0FF9A
:105FD000002F80CE05D1361F37601527FFF71EFE34
:105FE000F4E700BFFFF7CEFF18480568002D1AD16F
:105FF000FFF732FE042F06D104201449086080CE3A
:10600000FFF7D8FE0FE0182F06D118200F490860BF
:1060100080CEFFF7CFFE06E0012F03D180CEFFF741
:106020004FFF00E080CE09480568002DDAD0074810
:106030000568042DEFF3008001B4361F37602F464A
:1060400001BC80F3008800D1002700BD300A002089
:106050002C0A0020280A0020240A0020200A002000
:10606000074805688020054000B508D0054D064862
:10607000686006486860802029698143296100BD05
:10608000102002400020024023016745AB89EFCD7C
:10609000083E134931607760124F00B53068451EE5
:1060A000002DEFF3008001B4356001BC80F300885F
:1060B00004D0FD6801200540002DEFD1FD68342497
:1060C0002C40FC6030680028EFF3008001B42F46BC
:1060D000361D01BC80F3008801D10348074300BD91
:1060E00000001000002002400000008000B5FFF713
:1060F000B7FF084901200D6805430D6030683880FE
:1061000077680836FFF7C4FF024901200D68854310
:106110000D6000BD102002400B483F1A00B5FFF78C
:106120009FFF0A4D02202969014329616F614020C8
:1061300029690143296180CEFFF7AAFF04490220A3
:106140000D6885430D6000BD00000008002002407E
:106150001020024000B500BFFFF71BFD340A0020ED
:10616000202F80CE00B503D002490868401C08608B
:1061700000BD0000340A002030683F1830683760E6
:10618000074600B5FFF7FCFC93060020009D019830
:106190000544361F37602F46FFF7BEFFFFF7E0FFCD
:1061A00003480568009840190090EFD703B000BD80
:1061B0001400002005480568083E054931607760F5
:1061C0002F4600B5FFF7D8FF00BD000010000020EB
:1061D000000000087068054601218D4330680446C0
:1061E00001218C437F1C01218F433F19376075606B
:1061F000274600B5FFF7C4FC050700203D88009C3A
:1062000001980444083E356077602746FFF76EFF2B
:10621000FFF7A6FFBF1C0098801C0090EED703B0CC
:1062200080CE00BD361F3760802700B5FFF7D2FF54
:1062300000BD20200F200740092F00B500DDFF1D05
:106240003037FFF7EBFC00BD3D0B361F37602F46A4
:1062500000B5FFF7EFFF3D0A361F37602F46FFF707
:10626000E9FF3D09361F37602F46FFF7E3FFFFF7D1
:10627000E1FF00BD0845726173696E672006206406
:106280006F6E652010537461727420586D6F646571
:106290006D20545820265072657373205220746FFD
:1062A000207265626F6F742C206F74686572207441
:1062B0006F20726570726F6772616D200645727231
:1062C0006F7273034E6F20207D1C3F78361F356040
:1062D00000B5FFF7D9FC00BD00B5FFF7EFFC9C4D02
:1062E000361F37602F46FFF7AFFF361F3760202776
:1062F000FFF794FC361F3760014FFFF7E5FF00BD45
:10630000A007002000B5FFF775FC361F3760322765
:10631000FFF708FD00BD202000B5FFF7F3FF00BF29
:10632000284900200860FFF7C9FC361F3760264F58
:10633000FFF7CAFF361F37601427FFF7F3FCFFF79C
:1063400039FF361F3760214FFFF7BEFFFFF7C4FF4D
:106350001C4900200860FFF7B1FC361F37601C4F56
:10636000FFF7B2FF361F37601A27FFF757FC1948AF
:106370000568083E1849316077602F46FFF710FE28
:1063800080CEFFF7A9FF361F37606427FFF7CAFCEE
:10639000FFF794FC361F3760104FFFF795FFFFF7AC
:1063A0005BFCDF200740361F3760FFF737FC522FBA
:1063B00080CEB5D1361F37606427FFF7B3FCFFF7F7
:1063C000BBFC00BD340A00205807002061070020F4
:1063D0006807002010000020000000087907002056
:1063E00005436F707920202000B5FFF78BFFFFF782
:1063F00065FC361F3760174FFFF766FF361F3760A3
:106400001427FFF78FFC144900200860083EB1688C
:1064100031607760FFF7B0FEFFF75EFF361F376031
:106420000A27FFF77FFC4A4D002D02D0B7680C36D3
:1064300000BDFFF743FC361F3760084FFFF744FFEE
:10644000FFF7C8FEFFF748FF361F37601427FFF736
:1064500069FC00BD58070020340A0020C408002051
:1064600000B500BF0C3EF168316031697160B76002
:10647000FFF7BAFF364D002DF4D1361F3760642781
:10648000FFF750FCFFF758FC00BD000098570008CC
:10649000CB5245464C4153485541525400B500BF7C
:1064A000FBF74AF8AC1000202C590008C643414CB9
:1064B0004C49542072B60F480568103E0E493160B1
:1064C0000E497160B560F7600D4F00B5FAF73AFC00
:1064D000094DAF600B48E8600B4828610B486861C4
:1064E00035687768083601200543A847FDF7C6FBE5
:1064F00000BD0000AC100020000000201C5B000864
:1065000070090000006CDC0200F8010000080000C7
:10651000AC640008C75245464C41534804480568DE
:10652000361F37602F4600B5FFF7C4FF00BD0000DF
:106530001C5B0008045B0008C9434F5059464C419E
:106540005348202004480568361F37602F4600B5A1
:10655000FFF7B0FF00BD0000205B0008BC5800083A
:10656000CA4449534B2D4552524F522000B500BFEB
:10657000FAF7E2FFB010002090640008C8454E44CE
:106580002D4C4F41442020205D460020E8625D46AE
:10659000012040422863704700B500BFFBF746FE6C
:1065A000062F80CEFAD100BD361F3760002700B518
:1065B00080CEFBF73BFE152F01D0002501E0012521
:1065C0006D42062F01D0002701E001277F422F43B3
:1065D000EFF3008001B42F4601BC80F30088E7D0C0
:1065E00000BD2020361F376000B5FBF73BFE3F0A99
:1065F000FBF738FEFFF7D0FF00BD202000B500BF3D
:10660000FBF714FE012F80CEFAD100BFFBF71CFE72
:10661000002F80CE03D0FBF709FE80CEF6E7361FB1
:1066200037600627FBF71EFE00BD202000B5FBF7F4
:1066300019FEFFF7E3FF7D1C3F78083E3760756069
:10664000FFF7D0FFFBF720FE361F37600627FBF76A
:1066500009FEFFF7A9FF02490F6080CE00BD0000D0
:10666000B0100020361F3760052700B5FBF7FAFD94
:10667000FBF71AFEFCF74CF8084572726F72202384
:1066800020000000FCF760F9FBF70EFEFFF77CFF2F
:1066900000BD00007C6500088A53484F574C494EA6
:1066A00045533F2000B500BFFAF7F7FFB4100020B4
:1066B000361F3760062700B5FFF7B8FF361F376073
:1066C0001D4FFFF78FFF361F37600127FFF78AFF47
:1066D000FFF794FF5D46002028635D46012040429D
:1066E000E862002015490860FCF70AFFFCF77EFB12
:1066F00013480568002D05D0FBF7D6FDFCF766FBB7
:10670000FBF7C2FD361F37600E4FFCF70DF8002F68
:1067100000D180CE0AD0FFF7A5FF5D46AD69361FD8
:1067200037602F463E1C80CEFCF7EAFE5D462D6B9F
:10673000002DDBD000BD01B4FFFFFFFF941000204F
:10674000B4100020E8360008F0500008C7494E4356
:106750004C554445361F3760202700B5FCF7D4FB65
:106760007D1C3C78083E356077602746FAF752FB7F
:10677000FFF79EFF00BD0000E4550008C847454EE6
:10678000535049425220202030683760074600B5F8
:10679000FAF71AF8083E002131607760072700BF3A
:1067A000F9F79EFECB670008009D0198054401247F
:1067B000AC40BC4204DA009F0198074403B000BD1E
:1067C0000098401E0090EFD703B0002700BD0000E6
:1067D00064570008C928494E49545350492920207C
:1067E00000B580B4009F402039688143396080CE75
:1067F000FFF7CAFFFF0007480743009D2F60009F77
:106800000548786080BC402039680143396080CEFB
:1068100000BD000007030000001700004C670008DF
:10682000CD535049325F4E43535F4D454D53202069
:1068300000B500BFFAF743FE3C68000800080048B6
:106840000100000040000000F8570008C8535049FC
:10685000325F53434B20202000B500BFFAF72FFED4
:106860006468000800040048002000002D000000BB
:1068700038650008C9535049325F4D49534F2020B5
:1068800000B500BFFAF71BFE8C6800080004004842
:10689000004000002E00000074680008C9535049F1
:1068A000325F4D4F5349202000B500BFFAF707FE75
:1068B000B468000800040048008000002F000000B9
:1068C000D4670008C8495353504950494E202020EE
:1068D000083E00213160776000B5FEF7DDFB361F12
:1068E00003213160FEF76AFC00BD000098660008D5
:1068F000CA53454C494F2D5350493220174D184C1F
:10690000696921436961A96AA143A962134D154CC4
:10691000E9692143E9612969A1432961124D083ED2
:10692000356077602F4600B5FEF7A6FB083E0121D3
:1069300031607760FEF742FCFEF7BCFA361F376025
:106940000A4FFFF7C5FF361F3760094FFFF7C0FF3B
:10695000361F3760074FFFF7BBFF00BD0010024036
:106960000000C000004000003C68000864680008A7
:106970008C680008B468000890510008C75350495B
:106980005843484730683873361D00B5FAF710FB96
:10699000FAF70EFBFAF70CFBFAF70AFBBD68832047
:1069A0000540032DFAD13F7BFF20074000BD0000CA
:1069B0004C680008C8535049464C55534820202085
:1069C000361F3760044F00BFBD680120054001D06D
:1069D000FD68F9E780CE704700380040CC560008CB
:1069E000C453504921202020361F3760024F00B584
:1069F000FFF7C8FF80CE00BD00380040E069000806
:106A0000C453504940202020083EFF213160776068
:106A1000024F00B5FFF7B6FF00BD00000038004090
:106A2000C4680008C8494E495453504932202020B8
:106A300000B5FFF763FF0C3E054931600549716001
:106A4000B760054FFFF7CCFEFFF7BAFF00BD0000AF
:106A5000006CDC0240420F0000380040485900083A
:106A6000C52E535049322020083E044931607760DA
:106A7000402700B5FEF73CF900BD0000003800409B
:106A8000B4690008C853504944454C41592020205E
:106A9000361F3760092700BF7F1E002FFCD180CE34
:106AA000704700009C680008C943534C4F5F4D4538
:106AB0004D53202000B5FFF7EBFF361F3760034F23
:106AC000FEF704FAFFF7E4FF00BD00003C68000891
:106AD000A86A0008C9435348495F4D454D532020DB
:106AE00000B5FFF7D5FF361F3760034FFEF7E2F919
:106AF000FFF7CEFF00BD00003C680008E459000825
:106B0000C94D454D535F494E5431202000B500BF5B
:106B1000FAF7D5FC186B00080008004802000000D6
:106B200041000000006B0008C94D454D535F494EC0
:106B30005432202000B500BFFAF7C1FC406B0008BA
:106B4000000800480400000042000000146500082E
:106B5000CD4C33474432305F5752495445312020A1
:106B600000B5FFF7A7FF3F200740FFF73DFFFFF706
:106B70003BFFFFF7B5FF00BDD8580008CC4C3347AA
:106B80004432305F524541443120202000B5FFF7A8
:106B900091FF3F20074080200743FFF725FFFFF7C5
:106BA00033FFFFF79DFF00BD7C6B0008CC4C3347E3
:106BB0004432305F524541444E2020203068002846
:106BC00000B502D1B7680C3600BDFFF773FF3F2058
:106BD0000740C0200743FFF707FF30683F183068C1
:106BE00037600746F9F77CFC056C0008FFF70CFFDF
:106BF000009D019805442F7080CE0098401C0090A5
:106C0000F4D703B0FFF76CFF00BD0000D46A0008A2
:106C1000C95345544D41534B4C332020361F7168A6
:106C20003160776000B5FFF7B1FF3068C5433D4084
:106C3000B06805437768B5600836FFF791FF00BD7F
:106C4000006A0008C5424F524C332020361F71683D
:106C5000316000B5FFF7E2FF00BD0000AC6B00083B
:106C6000C6424249434C3320361F716831600021CF
:106C7000716000B5FFF7D2FF00BD0000106C000886
:106C8000D04C33474432305F5245424F4F54434D0E
:106C900044202020083E802131607760242700B501
:106CA000FFF7D4FF00BD000020680008D44C334734
:106CB0004432305F47455444415441535441545544
:106CC00053202020361F3760272700B5FFF75EFFCF
:106CD00000BD0000A8590008CB494E49542D4C3343
:106CE0004744323000B5FFF7A3FE1E4D083E356025
:106CF00077602F46FEF7B0F9FEF730FA1A4D083EDE
:106D0000356077602F46FEF7A7F9FEF727FA083EB1
:106D10000F21316077602027FFF722FF083E002116
:106D2000316077602127FFF71BFF083E00213160AB
:106D300077602227FFF714FF083E902131607760CB
:106D40002327FFF70DFF083E40213160776024279D
:106D5000FFF706FF083E0021316077602E27FFF71E
:106D6000FFFE00BD186B0008406B0008606A000859
:106D7000D74C33474432305F494E5431494E544525
:106D80005252555054434D44002F01D1002701E089
:106D900001277F4280200740083E802131607760D4
:106DA000222700B5FFF73AFF00BD0000706D000814
:106DB000D74C33474432305F494E5432494E5445E4
:106DC0005252555054434D44002F01D1002701E049
:106DD00001277F4208200740083E08213160776084
:106DE000222700B5FFF71AFF00BD0000286B00083E
:106DF000C2545220361F37600F2700B5FFF7C6FE7A
:106E0000FDF796FE00BD0000506B0008C8415849D0
:106E1000534441544120202000B500BFFAF74FFBF6
:106E2000000200207C690008C85245414441584591
:106E30005320202000B500BF361F37602727FFF7FB
:106E4000A5FE0820074080CEF6D00C3E062131601A
:106E500003497160B7602827FFF7B0FE00BD00004E
:106E600000020020B06D0008C52E41584553202077
:106E700000B5FBF719FA361F3760164FFBF748FCD1
:106E80000458203D2000000000217D5E361F376041
:106E90002F46FBF759FDBF1CFBF73AFC0459203D78
:106EA0002000000000217D5E361F37602F46FBF773
:106EB0004BFDBF1CFBF72CFC045A203D20000000BA
:106EC00000217D5E361F37602F46FBF73DFDBF1C5E
:106ED00080CE00BD00020020286E0008C852454147
:106EE000445445535420202000B5FFF7FBFE00BF5B
:106EF000FFF7A0FFFFF7BCFF361F37606427FEF7E0
:106F0000EDFAFBF7A1F9002F80CEF1D000BD000013
:106F10007C670008CA55534552425554544F4E2081
:106F200000B500BFFAF7CBFA2C6F0008000000484C
:106F30000100000000000000686E0008C74C4544D6
:106F4000534F4646361F3760094F00B5FDF7BEFF69
:106F5000361F3760074FFDF7B9FF361F3760064F02
:106F6000FDF7B4FF361F3760044FFDF7AFFF00BDDC
:106F700084520008E4520008C4520008A4520008D9
:106F8000806C0008C45856414C2020200348002142
:106F9000455E361F37602F46704700000002002014
:106FA000F0680008C45956414C20202003480021B5
:106FB000455E361F37602F467047000002020020F2
:106FC00060650008C45A56414C2020200348002127
:106FD000455E361F37602F467047000004020020D0
:106FE000F06D0008C74F4E4C594C454400B5FFF7B3
:106FF000A9FFFDF75FFF361F3760FA27FEF76EFA2D
:1070000000BD0000846F0008C844454D4F4D454DFC
:107010005320202000B5FBF747F9FBF779FB2C54F0
:107020006865204C4544732077696C6C20666F6CF2
:107030006C6F7720746865206D6F74696F6E206F58
:10704000662074686520626F61726400FBF72CF93A
:10705000FBF75EFB1F756E74696C20796F7520708D
:1070600072657373207468652055534552206275AC
:1070700074746F6E354900200860FFF763FFFFF7F7
:1070800031FE361F3760324FFDF7E6FFFFF7D2FEC5
:10709000FFF77CFF002F00D57F42FFF787FF002F0F
:1070A00000D57F4230688742EFF3008001B47768F3
:1070B000083601BC80F3008815DAFFF767FF282F38
:1070C00080CE04DD361F3760224FFFF78FFFFFF7BA
:1070D0005DFF2820C74280CE04DA361F37601E4F7E
:1070E000FFF784FF14E0FFF761FF282F80CE04DD57
:1070F000361F3760194FFFF779FFFFF757FF28203A
:10710000C74280CE04DA361F3760154FFFF76EFF97
:10711000FAF700FC361F37600D4FFDF7E3FE002F36
:1071200080CEB3D0FAF7F6FB361F3760084FFDF775
:10713000D9FE002F80CEF5D1FFF704FF03490120CF
:1071400040420860FBF7B0F800BD00009C10002032
:107150002C6F0008A4520008E45200088452000872
:10716000C4520008606C0008C652502D454E4420A1
:1071700000B500BFFAF7A3F900400020B8000000F6
:1071800000100020000000000000000000000000CF
:1071900000000000B00F000800000000E800000040
:1071A0000000000000000000000000001810002097
:1071B00000000000000000000000000000000000CF
:1071C00000000000B00F000800000000BC21000813
:1071D00010000000AC6C0008246A00085456000837
:1071E0003C6F0008D86C000824520008E46F0008C7
:1071F000446C0008687100080C6E0008DC6E000822
:10720000846A000808700008A46F0008C46F0008B2
:10721000146F000800000000AC2B00080000000004
:10722000EC57000801000000000000000000000012
:10723000DC5500080038014000000000000000009C
:10724000000000000000000000000000000000003E
:00000001FF
